:020000020000FC
:100000000C945C040C942A000C942A000C942A0092
:100010000C942A000C942A000C942A000C942A00B8
:100020000C942A000C942A000C94B9000C942A0019
:100030000C942A000C942A000C942A000C942A0098
:100040000C942A000C942A000C942A000C942A0088
:100050000C942A0018959198899A0895919A899AF2
:100060000895919BFBCFF7CFA0E6B0E6EAE2F0E07F
:10007000ED93FD93E0E0F0E0ED93FD930895FF91A3
:10008000EF91EE0FFF1F8F939F9385919591A0E6BF
:10009000B0E01D900D90911538F011F0C00104C032
:1000A000801510F009F0C0018D939D9305910D937B
:1000B0000197E1F79F918F91E0FB0EF43196F69551
:1000C000E79509940F730D9308950D9108950930E4
:1000D00008F40EE20F3708F00EE200FB069507F970
:1000E0000D9308958F939F93E0E6F0E0329681910F
:1000F00091910C910F3B29F00191E9DF81509040E3
:10010000C1F79F918F9108953F934F93AEE8B0E070
:100110003EE103E0D7DF0BE1D5DF0FE0D3DF0FE3F4
:10012000D1DF0CE3CFDF48E20EE2D1DF4A95E1F701
:100130000FEB0D933A9569F74F913F9108956A95AA
:10014000F1F70895AE98AF98A69AA79A979A8F98C4
:100150000895AE9A67E0F3DFAE9808951F012D0170
:1001600062E068BFFF91EF91BF91AF916F916FBF58
:1001700018956FB76F93AF93BF93EF93FF93000002
:10018000000000000000000062B7623001F00000D3
:1001900000000000000062B7633001F000000000C2
:1001A0000000000062B7643001F0D201F10109944F
:1001B000F8946FB76F93AF93BF93EF93FF9360E0A3
:1001C00062BF6AE46CBF6AE063BF62E069BF87999F
:1001D0006CE0879B6CE0662E6FEF762EBADFE2EF65
:1001E000F0E0BCCF62E0ABDF00006A9449F00000B1
:1001F0000000000000000000000000000000EECF42
:1002000087996DE0879B6DE0662E6EEF762EAF9A34
:10021000A0DFECE0F1E0A2CF62E091DF00006A94A1
:1002200049F0000000000000000000000000000095
:100230000000EECF879969E1879B69E1662E6DEF3B
:10024000762EAF9886DFE6E2F1E088CF62E077DFD6
:100250006A94D9F0000000000000000000000000D7
:10026000000000000000EECF0FEF7016F1F37016E3
:10027000F1F7089500E0802E85BA04B30F6304BB44
:10028000969A8E98959A8D980895AEE8B0E08799E1
:1002900069E1879B6EE1762E70E060E0662E59DFA3
:1002A00060FE11C0869B11C09C908599982C9E96EB
:1002B0006CE045DF0000000095BAE0E6F1E04ECFCB
:1002C00085BA0C9473010000000068E038DF00007C
:1002D0009D90AD90DD90CD90BD90ED91FE2FFF7380
:1002E000E078E72B0994609421F09E9763E027DF84
:1002F000D6CF705F707731F09E9761E020DF00000D
:100300000000CDCF7A9429F4000000000000000026
:100310005ECF0000000000000000000000000000B0
:10032000000000000000BBCF3E3160F4153050F4F7
:10033000AEE8B0E02EE2329FA00DB11DA10F20E08B
:10034000B21FC0CE08953E31E8F71530D8F7AEE8B9
:10035000B0E02EE2329FA00DB11DA10F20E0B21F30
:10036000B4CE3E3178F7483268F7A3E9B0E02EE228
:10037000329FA00DB11DA40F20E0B21FA8CE3E31C8
:1003800008F74832F8F6A3E9B0E02EE2329FA00D5C
:10039000B11DA40F20E0B21FA5CEF1DF3395089563
:1003A0004F9340E06CDE28002020202020202020D9
:1003B000202020202020202020202020202020203D
:1003C000202020202020202020202020202020202D
:1003D000E4DF4F91089553DE2000202122232425BD
:1003E000262728292A2B2C2D2E2F30313233343535
:1003F000363738393A3B3C3D3E3FCFDF40DE2000C8
:10040000404142434445464748494A4B4C4D4E4F74
:10041000505152535455565758595A5B5C5D5E5F64
:10042000BCDF2DDE20006061626364656667686919
:100430006A6B6C6D6E6F70717273747576777879A4
:100440007A7B7C7D7E20A9DF0895AADFA9DFA8DF63
:1004500033504F9344E0BFDF4F91089500E010E028
:1004600063DF9ECF10E060DF00E011E05DDF3395D9
:10047000089500E3F7DF0CE3F5DF0CE0F3DF0FE0B6
:10048000F1DF03E0EFDF03E3EDDF36500895F7DD42
:1004900017002D275F5F602D2E5F5F2E2D275F5F7A
:1004A000602D2E5F5F2E2D275F2077DF0895EFDF11
:1004B000EEDFEDDFECDFEBDFEADF08950FE151DF88
:1004C00033950895FBDFFADFF9DFF8DFF7DFF6DFBA
:1004D0000895D5DD1000101C1C1C1C1C1C1C1C1CB1
:1004E0001C1C1C1C1C1059DFCADD10001018141035
:1004F00010101418101818101C1014104EDFBFDD47
:10050000100010191018101E141E141A1A1A101A9E
:100510001A1043DFB4DD100010101515151A101A4B
:100520001012161A1A1A1B1038DFA9DD100010134A
:1005300010121012101011101110131212102DDFC2
:100540009EDD10001013131313131313131313133F
:100550001313131022DF0895AADF3650495EB2DF6D
:1005600036504F5FB6DF4851089589DD2800415469
:100570006D656761333220415652207543202B2030
:10058000536F6674564741203D203430306C696E9D
:1005900065203730487A01DF72DD280031382E348B
:1005A00033324D487A2C2033636C6B2F7069786C32
:1005B0002C20347069786C2F636861722C20343081
:1005C00063686172EADE5BDD280034783870697830
:1005D000656C20666F6E742C203935204153434979
:1005E000492C20313620626C6F636B6772617068D2
:1005F0006963D3DE08950F9300E010E095DE0F915C
:100600000F9311E091DE0F910F930A7212E08CDECE
:100610000F910F93057113E087DE0F910A6214E0CA
:1006200083DE3395089503E0E6DF0CE0E4DF0FE0BE
:10063000E2DF00E3E0DF03E3DEDF0CE3DCDF0FE318
:10064000DADF375008951BDD28006E6F720E696E79
:10065000760F6E6F720C756C696E0D6E6F720B3269
:100660002F330B6E6F720A312F330A6E6F7209705F
:10067000617393DE0895E7DFE6DFE5DFE4DFE3DFC4
:10068000E2DFE1DF0895FBDC280064657369676ED3
:1006900020616E6420636F6465206F70656E2073E7
:1006A0006F7572636520617661696C61626C65204B
:1006B000617473DEE4DC2800687474703A2F2F6E66
:1006C00065696C2E6672616E6B6C696E2E63682F45
:1006D00050726F6A656374732F536F667456474127
:1006E0005CDE08953F934F9330E040E0AEDEB6DE2F
:1006F000C0DE32DFB3DE39DFB1DE95DFBCDFAEDE78
:10070000C2DFACDE4F913F91089510E01CDE005F28
:100710000BDE0895949A8C9884990895052F0F7391
:1007200041F43F9330E0F1DF3395EFDF3395EDDFB8
:100730003F9108953F934F9336E14091F2059FDC3E
:1007400004002020202029DE3150939A8B98839931
:100750000EC0052F0F7031F44395483208F040E089
:100760004093F2058CDC04005F405F2F16DE4F9152
:100770003F91089584DC06002020202020200DDEFB
:100780000895F8DFF7DFF6DFF5DFF4DFF3DF089534
:1007900076DC03002E2D2E2000DE71DC03007C2091
:1007A0007C20FBDD6CDC0300602D2720F6DD089546
:1007B00066DC03002E2D1010F0DD61DC03007C20D0
:1007C0001510EBDD5CDC0300602D1010E6DD0895F4
:1007D00056DC03002E1C1010E0DD51DC03007C1001
:1007E0001510DBDD4CDC030060131010D6DD08951E
:1007F00046DC0300101C1010D0DD41DC03001A1091
:100800001510CBDD3CDC030010131010C6DD08957D
:10081000123018F410FFBCCFCBCF10FFD9CFE8CFE8
:100820003F934F9334E040E042DE3650929A8A98EC
:1008300082991CC040E146DE36504395A2DF365017
:10084000052F069506950695102F077027E002FDE7
:10085000201B02FD022F300F16951395177027E00D
:1008600012FD211B12FD122F410FD2DF4F913F913C
:1008700008953F934F933BE040E077DE3350919AE9
:10088000899881990DC050FF0BC0052F06950695DC
:100890000695069500FF04C00695400F0FE561DD43
:1008A0004F913F9108951EDF50E0DEDC539532DF1B
:1008B00041DFB6DFDEDFF9CFEFE5F8E0EDBFFEBFE9
:0E08C0007894D2DB21DC3EDCD5DC72DCECCFA0
:1009000095BAAB24BA24AB24ED91FE2FFF73E078A7
:10091000E06009943031323334353637383930318C
:1009200095BAAB24BA24AB24ED91FE2FFF73E07887
:10093000E06109943031323334353637383930316B
:1009400095BAAB24BA24AB24ED91FE2FFF73E07867
:10095000E06209943031323334353637383930314A
:1009600095BAAB24BA24AB24ED91FE2FFF73E07847
:10097000E063099430313233343536373839303129
:1009800095BAAB24BA24AB24ED91FE2FFF73E07827
:10099000E064099430313233343536373839303108
:1009A00095BAAB24BA24AB24ED91FE2FFF73E07807
:1009B000E0650994303132333435363738393031E7
:1009C00095BAAB24BA24AB24ED91FE2FFF73E078E7
:1009D000E0660994303132333435363738393031C6
:1009E00095BAAB24BA24AB24ED91FE2FFF73E078C7
:1009F000E0670994303132333435363738393031A5
:100A000095BAAC24CA24AC24ED91FE2FFF73E07894
:100A1000E06009943031323334353637383930318B
:100A200095BAAC24CA24AC24ED91FE2FFF73E07874
:100A3000E06109943031323334353637383930316A
:100A400095BAAC24CA24AC24ED91FE2FFF73E07854
:100A5000E062099430313233343536373839303149
:100A600095BAAC24CA24AC24ED91FE2FFF73E07834
:100A7000E063099430313233343536373839303128
:100A800095BAAC24CA24AC24ED91FE2FFF73E07814
:100A9000E064099430313233343536373839303107
:100AA00095BAAC24CA24AC24ED91FE2FFF73E078F4
:100AB000E0650994303132333435363738393031E6
:100AC00095BAAC24CA24AC24ED91FE2FFF73E078D4
:100AD000E0660994303132333435363738393031C5
:100AE00095BAAC24CA24AC24ED91FE2FFF73E078B4
:100AF000E0670994303132333435363738393031A4
:100B000095BAAD24DA24AD24ED91FE2FFF73E07881
:100B1000E06009943031323334353637383930318A
:100B200095BAAD24DA24AD24ED91FE2FFF73E07861
:100B3000E061099430313233343536373839303169
:100B400095BAAD24DA24AD24ED91FE2FFF73E07841
:100B5000E062099430313233343536373839303148
:100B600095BAAD24DA24AD24ED91FE2FFF73E07821
:100B7000E063099430313233343536373839303127
:100B800095BAAD24DA24AD24ED91FE2FFF73E07801
:100B9000E064099430313233343536373839303106
:100BA00095BAAD24DA24AD24ED91FE2FFF73E078E1
:100BB000E0650994303132333435363738393031E5
:100BC00095BAAD24DA24AD24ED91FE2FFF73E078C1
:100BD000E0660994303132333435363738393031C4
:100BE00095BAAD24DA24AD24ED91FE2FFF73E078A1
:100BF000E0670994303132333435363738393031A3
:100C000095BA000000000000ED91FE2FFF73E07820
:100C1000E060099430313233343536373839303189
:100C200095BA000000000000ED91FE2FFF73E07800
:100C3000E061099430313233343536373839303168
:100C400095BA000000000000ED91FE2FFF73E078E0
:100C5000E062099430313233343536373839303147
:100C600095BA000000000000ED91FE2FFF73E078C0
:100C7000E063099430313233343536373839303126
:100C800095BA000000000000ED91FE2FFF73E078A0
:100C9000E064099430313233343536373839303105
:100CA00095BA000000000000ED91FE2FFF73E07880
:100CB000E0650994303132333435363738393031E4
:100CC00095BA000000000000ED91FE2FFF73E07860
:100CD000E0660994303132333435363738393031C3
:100CE00095BAA9249A24A924ED91FE2FFF73E078E8
:100CF000E0670994303132333435363738393031A2
:100D000095BA000000000000ED91FE2FFF73E0781F
:100D1000E060099430313233343536373839303188
:100D200095BA000000000000ED91FE2FFF73E078FF
:100D3000E061099430313233343536373839303167
:100D400095BA000000000000ED91FE2FFF73E078DF
:100D5000E062099430313233343536373839303146
:100D600095BA000000000000ED91FE2FFF73E078BF
:100D7000E063099430313233343536373839303125
:100D800095BA000000000000ED91FE2FFF73E0789F
:100D9000E064099430313233343536373839303104
:100DA00095BA000000000000ED91FE2FFF73E0787F
:100DB000E0650994303132333435363738393031E3
:100DC00095BA000000000000ED91FE2FFF73E0785F
:100DD000E0660994303132333435363738393031C2
:100DE000A5BAA9249A24A924ED91FE2FFF73E078D7
:100DF000E0670994303132333435363738393031A1
:100E000095BAA9249A24A924ED91FE2FFF73E078C6
:100E1000E060099430313233343536373839303187
:100E200095BAA9249A24A924ED91FE2FFF73E078A6
:100E3000E061099430313233343536373839303166
:100E400095BAA9249A24A924ED91FE2FFF73E07886
:100E5000E062099430313233343536373839303145
:100E600095BAA9249A24A924ED91FE2FFF73E07866
:100E7000E063099430313233343536373839303124
:100E800095BAA9249A24A924ED91FE2FFF73E07846
:100E9000E064099430313233343536373839303103
:100EA00095BAA9249A24A924ED91FE2FFF73E07826
:100EB000E0650994303132333435363738393031E2
:100EC00095BAA9249A24A924ED91FE2FFF73E07806
:100ED000E0660994303132333435363738393031C1
:100EE00095BAA9249A24A924ED91FE2FFF73E078E6
:100EF000E0670994303132333435363738393031A0
:100F0000A5BAA9249A24A924ED91FE2FFF73E078B5
:100F1000E060099430313233343536373839303186
:100F2000A5BAA9249A24A924ED91FE2FFF73E07895
:100F3000E061099430313233343536373839303165
:100F4000A5BAA9249A24A924ED91FE2FFF73E07875
:100F5000E062099430313233343536373839303144
:100F6000A5BAA9249A24A924ED91FE2FFF73E07855
:100F7000E063099430313233343536373839303123
:100F8000A5BAA9249A24A924ED91FE2FFF73E07835
:100F9000E064099430313233343536373839303102
:100FA000A5BAA9249A24A924ED91FE2FFF73E07815
:100FB000E0650994303132333435363738393031E1
:100FC000A5BAA9249A24A924ED91FE2FFF73E078F5
:100FD000E0660994303132333435363738393031C0
:100FE000A5BAA9249A24A924ED91FE2FFF73E078D5
:100FF000E06709943031323334353637383930319F
:1010000095BAED9195BAFE2FFF7395BAE078E0603E
:1010100095BA099430313233343536373839303176
:1010200095BAED9195BAFE2FFF7395BAE078E0611D
:1010300095BA099430313233343536373839303156
:1010400095BAED9195BAFE2FFF7395BAE078E062FC
:1010500095BA099430313233343536373839303136
:1010600095BAED9195BAFE2FFF7395BAE078E063DB
:1010700095BA099430313233343536373839303116
:1010800095BAED9195BAFE2FFF7395BAE078E064BA
:1010900095BA0994303132333435363738393031F6
:1010A00095BAED9195BAFE2FFF7395BAE078E06599
:1010B00095BA0994303132333435363738393031D6
:1010C00095BAED9195BAFE2FFF7395BAE078E06678
:1010D00095BA0994303132333435363738393031B6
:1010E00095BAED9195BAFE2FFF7395BAE078E06757
:1010F00095BA099430313233343536373839303196
:10110000A5BAED91A5BAFE2FFF7395BAE078E0601D
:1011100095BA099430313233343536373839303175
:10112000A5BAED91A5BAFE2FFF7395BAE078E061FC
:1011300095BA099430313233343536373839303155
:10114000A5BAED91A5BAFE2FFF7395BAE078E062DB
:1011500095BA099430313233343536373839303135
:10116000A5BAED91A5BAFE2FFF7395BAE078E063BA
:1011700095BA099430313233343536373839303115
:1011800095BAED9195BAFE2FFF7395BAE078E064B9
:1011900095BA0994303132333435363738393031F5
:1011A00095BAED9195BAFE2FFF7395BAE078E06598
:1011B00095BA0994303132333435363738393031D5
:1011C00095BAED9195BAFE2FFF7395BAE078E06677
:1011D00095BA0994303132333435363738393031B5
:1011E00095BAED9195BAFE2FFF7395BAE078E06756
:1011F00095BA099430313233343536373839303195
:1012000095BAED9195BAFE2FFF73A5BAE078E0602C
:10121000A5BA099430313233343536373839303164
:1012200095BAED9195BAFE2FFF73A5BAE078E0610B
:10123000A5BA099430313233343536373839303144
:1012400095BAED9195BAFE2FFF73A5BAE078E062EA
:10125000A5BA099430313233343536373839303124
:1012600095BAED9195BAFE2FFF73A5BAE078E063C9
:10127000A5BA099430313233343536373839303104
:1012800095BAED9195BAFE2FFF7395BAE078E064B8
:1012900095BA0994303132333435363738393031F4
:1012A00095BAED9195BAFE2FFF7395BAE078E06597
:1012B00095BA0994303132333435363738393031D4
:1012C00095BAED9195BAFE2FFF7395BAE078E06676
:1012D00095BA0994303132333435363738393031B4
:1012E00095BAED9195BAFE2FFF7395BAE078E06755
:1012F00095BA099430313233343536373839303194
:10130000A5BAED91A5BAFE2FFF73A5BAE078E0600B
:10131000A5BA099430313233343536373839303163
:10132000A5BAED91A5BAFE2FFF73A5BAE078E061EA
:10133000A5BA099430313233343536373839303143
:10134000A5BAED91A5BAFE2FFF73A5BAE078E062C9
:10135000A5BA099430313233343536373839303123
:10136000A5BAED91A5BAFE2FFF73A5BAE078E063A8
:10137000A5BA099430313233343536373839303103
:1013800095BAED9195BAFE2FFF7395BAE078E064B7
:1013900095BA0994303132333435363738393031F3
:1013A00095BAED9195BAFE2FFF7395BAE078E06596
:1013B00095BA0994303132333435363738393031D3
:1013C00095BAED9195BAFE2FFF7395BAE078E06675
:1013D00095BA0994303132333435363738393031B3
:1013E00095BAED9195BAFE2FFF7395BAE078E06754
:1013F00095BA099430313233343536373839303193
:1014000095BAED9195BAFE2FFF7395BAE078E0603A
:1014100095BA099430313233343536373839303172
:1014200095BAED9195BAFE2FFF7395BAE078E06119
:1014300095BA099430313233343536373839303152
:1014400095BAED9195BAFE2FFF7395BAE078E062F8
:1014500095BA099430313233343536373839303132
:1014600095BAED9195BAFE2FFF7395BAE078E063D7
:1014700095BA099430313233343536373839303112
:10148000A5BAED91A5BAFE2FFF7395BAE078E06496
:1014900095BA0994303132333435363738393031F2
:1014A000A5BAED91A5BAFE2FFF7395BAE078E06575
:1014B00095BA0994303132333435363738393031D2
:1014C000A5BAED91A5BAFE2FFF7395BAE078E06654
:1014D00095BA0994303132333435363738393031B2
:1014E000A5BAED91A5BAFE2FFF7395BAE078E06733
:1014F00095BA099430313233343536373839303192
:10150000A5BAED91A5BAFE2FFF7395BAE078E06019
:1015100095BA099430313233343536373839303171
:10152000A5BAED91A5BAFE2FFF7395BAE078E061F8
:1015300095BA099430313233343536373839303151
:10154000A5BAED91A5BAFE2FFF7395BAE078E062D7
:1015500095BA099430313233343536373839303131
:10156000A5BAED91A5BAFE2FFF7395BAE078E063B6
:1015700095BA099430313233343536373839303111
:10158000A5BAED91A5BAFE2FFF7395BAE078E06495
:1015900095BA0994303132333435363738393031F1
:1015A000A5BAED91A5BAFE2FFF7395BAE078E06574
:1015B00095BA0994303132333435363738393031D1
:1015C000A5BAED91A5BAFE2FFF7395BAE078E06653
:1015D00095BA0994303132333435363738393031B1
:1015E000A5BAED91A5BAFE2FFF7395BAE078E06732
:1015F00095BA099430313233343536373839303191
:1016000095BAED9195BAFE2FFF73A5BAE078E06028
:10161000A5BA099430313233343536373839303160
:1016200095BAED9195BAFE2FFF73A5BAE078E06107
:10163000A5BA099430313233343536373839303140
:1016400095BAED9195BAFE2FFF73A5BAE078E062E6
:10165000A5BA099430313233343536373839303120
:1016600095BAED9195BAFE2FFF73A5BAE078E063C5
:10167000A5BA099430313233343536373839303100
:10168000A5BAED91A5BAFE2FFF7395BAE078E06494
:1016900095BA0994303132333435363738393031F0
:1016A000A5BAED91A5BAFE2FFF7395BAE078E06573
:1016B00095BA0994303132333435363738393031D0
:1016C000A5BAED91A5BAFE2FFF7395BAE078E06652
:1016D00095BA0994303132333435363738393031B0
:1016E000A5BAED91A5BAFE2FFF7395BAE078E06731
:1016F00095BA099430313233343536373839303190
:10170000A5BAED91A5BAFE2FFF73A5BAE078E06007
:10171000A5BA09943031323334353637383930315F
:10172000A5BAED91A5BAFE2FFF73A5BAE078E061E6
:10173000A5BA09943031323334353637383930313F
:10174000A5BAED91A5BAFE2FFF73A5BAE078E062C5
:10175000A5BA09943031323334353637383930311F
:10176000A5BAED91A5BAFE2FFF73A5BAE078E063A4
:10177000A5BA0994303132333435363738393031FF
:10178000A5BAED91A5BAFE2FFF7395BAE078E06493
:1017900095BA0994303132333435363738393031EF
:1017A000A5BAED91A5BAFE2FFF7395BAE078E06572
:1017B00095BA0994303132333435363738393031CF
:1017C000A5BAED91A5BAFE2FFF7395BAE078E06651
:1017D00095BA0994303132333435363738393031AF
:1017E000A5BAED91A5BAFE2FFF7395BAE078E06730
:1017F00095BA09943031323334353637383930318F
:1018000095BAED9195BAFE2FFF7395BAE078E06036
:1018100095BA09943031323334353637383930316E
:1018200095BAED9195BAFE2FFF7395BAE078E06115
:1018300095BA09943031323334353637383930314E
:1018400095BAED9195BAFE2FFF7395BAE078E062F4
:1018500095BA09943031323334353637383930312E
:1018600095BAED9195BAFE2FFF7395BAE078E063D3
:1018700095BA09943031323334353637383930310E
:1018800095BAED9195BAFE2FFF73A5BAE078E064A2
:10189000A5BA0994303132333435363738393031DE
:1018A00095BAED9195BAFE2FFF73A5BAE078E06581
:1018B000A5BA0994303132333435363738393031BE
:1018C00095BAED9195BAFE2FFF73A5BAE078E06660
:1018D000A5BA09943031323334353637383930319E
:1018E00095BAED9195BAFE2FFF73A5BAE078E0673F
:1018F000A5BA09943031323334353637383930317E
:10190000A5BAED91A5BAFE2FFF7395BAE078E06015
:1019100095BA09943031323334353637383930316D
:10192000A5BAED91A5BAFE2FFF7395BAE078E061F4
:1019300095BA09943031323334353637383930314D
:10194000A5BAED91A5BAFE2FFF7395BAE078E062D3
:1019500095BA09943031323334353637383930312D
:10196000A5BAED91A5BAFE2FFF7395BAE078E063B2
:1019700095BA09943031323334353637383930310D
:1019800095BAED9195BAFE2FFF73A5BAE078E064A1
:10199000A5BA0994303132333435363738393031DD
:1019A00095BAED9195BAFE2FFF73A5BAE078E06580
:1019B000A5BA0994303132333435363738393031BD
:1019C00095BAED9195BAFE2FFF73A5BAE078E0665F
:1019D000A5BA09943031323334353637383930319D
:1019E00095BAED9195BAFE2FFF73A5BAE078E0673E
:1019F000A5BA09943031323334353637383930317D
:101A000095BAED9195BAFE2FFF73A5BAE078E06024
:101A1000A5BA09943031323334353637383930315C
:101A200095BAED9195BAFE2FFF73A5BAE078E06103
:101A3000A5BA09943031323334353637383930313C
:101A400095BAED9195BAFE2FFF73A5BAE078E062E2
:101A5000A5BA09943031323334353637383930311C
:101A600095BAED9195BAFE2FFF73A5BAE078E063C1
:101A7000A5BA0994303132333435363738393031FC
:101A800095BAED9195BAFE2FFF73A5BAE078E064A0
:101A9000A5BA0994303132333435363738393031DC
:101AA00095BAED9195BAFE2FFF73A5BAE078E0657F
:101AB000A5BA0994303132333435363738393031BC
:101AC00095BAED9195BAFE2FFF73A5BAE078E0665E
:101AD000A5BA09943031323334353637383930319C
:101AE00095BAED9195BAFE2FFF73A5BAE078E0673D
:101AF000A5BA09943031323334353637383930317C
:101B0000A5BAED91A5BAFE2FFF73A5BAE078E06003
:101B1000A5BA09943031323334353637383930315B
:101B2000A5BAED91A5BAFE2FFF73A5BAE078E061E2
:101B3000A5BA09943031323334353637383930313B
:101B4000A5BAED91A5BAFE2FFF73A5BAE078E062C1
:101B5000A5BA09943031323334353637383930311B
:101B6000A5BAED91A5BAFE2FFF73A5BAE078E063A0
:101B7000A5BA0994303132333435363738393031FB
:101B800095BAED9195BAFE2FFF73A5BAE078E0649F
:101B9000A5BA0994303132333435363738393031DB
:101BA00095BAED9195BAFE2FFF73A5BAE078E0657E
:101BB000A5BA0994303132333435363738393031BB
:101BC00095BAED9195BAFE2FFF73A5BAE078E0665D
:101BD000A5BA09943031323334353637383930319B
:101BE00095BAED9195BAFE2FFF73A5BAE078E0673C
:101BF000A5BA09943031323334353637383930317B
:101C000095BAED9195BAFE2FFF7395BAE078E06032
:101C100095BA09943031323334353637383930316A
:101C200095BAED9195BAFE2FFF7395BAE078E06111
:101C300095BA09943031323334353637383930314A
:101C400095BAED9195BAFE2FFF7395BAE078E062F0
:101C500095BA09943031323334353637383930312A
:101C600095BAED9195BAFE2FFF7395BAE078E063CF
:101C700095BA09943031323334353637383930310A
:101C8000A5BAED91A5BAFE2FFF73A5BAE078E0647E
:101C9000A5BA0994303132333435363738393031DA
:101CA000A5BAED91A5BAFE2FFF73A5BAE078E0655D
:101CB000A5BA0994303132333435363738393031BA
:101CC000A5BAED91A5BAFE2FFF73A5BAE078E0663C
:101CD000A5BA09943031323334353637383930319A
:101CE000A5BAED91A5BAFE2FFF73A5BAE078E0671B
:101CF000A5BA09943031323334353637383930317A
:101D0000A5BAED91A5BAFE2FFF7395BAE078E06011
:101D100095BA099430313233343536373839303169
:101D2000A5BAED91A5BAFE2FFF7395BAE078E061F0
:101D300095BA099430313233343536373839303149
:101D4000A5BAED91A5BAFE2FFF7395BAE078E062CF
:101D500095BA099430313233343536373839303129
:101D6000A5BAED91A5BAFE2FFF7395BAE078E063AE
:101D700095BA099430313233343536373839303109
:101D8000A5BAED91A5BAFE2FFF73A5BAE078E0647D
:101D9000A5BA0994303132333435363738393031D9
:101DA000A5BAED91A5BAFE2FFF73A5BAE078E0655C
:101DB000A5BA0994303132333435363738393031B9
:101DC000A5BAED91A5BAFE2FFF73A5BAE078E0663B
:101DD000A5BA099430313233343536373839303199
:101DE000A5BAED91A5BAFE2FFF73A5BAE078E0671A
:101DF000A5BA099430313233343536373839303179
:101E000095BAED9195BAFE2FFF73A5BAE078E06020
:101E1000A5BA099430313233343536373839303158
:101E200095BAED9195BAFE2FFF73A5BAE078E061FF
:101E3000A5BA099430313233343536373839303138
:101E400095BAED9195BAFE2FFF73A5BAE078E062DE
:101E5000A5BA099430313233343536373839303118
:101E600095BAED9195BAFE2FFF73A5BAE078E063BD
:101E7000A5BA0994303132333435363738393031F8
:101E8000A5BAED91A5BAFE2FFF73A5BAE078E0647C
:101E9000A5BA0994303132333435363738393031D8
:101EA000A5BAED91A5BAFE2FFF73A5BAE078E0655B
:101EB000A5BA0994303132333435363738393031B8
:101EC000A5BAED91A5BAFE2FFF73A5BAE078E0663A
:101ED000A5BA099430313233343536373839303198
:101EE000A5BAED91A5BAFE2FFF73A5BAE078E06719
:101EF000A5BA099430313233343536373839303178
:101F0000A5BAED91A5BAFE2FFF73A5BAE078E060FF
:101F1000A5BA099430313233343536373839303157
:101F2000A5BAED91A5BAFE2FFF73A5BAE078E061DE
:101F3000A5BA099430313233343536373839303137
:101F4000A5BAED91A5BAFE2FFF73A5BAE078E062BD
:101F5000A5BA099430313233343536373839303117
:101F6000A5BAED91A5BAFE2FFF73A5BAE078E0639C
:101F7000A5BA0994303132333435363738393031F7
:101F8000A5BAED91A5BAFE2FFF73A5BAE078E0647B
:101F9000A5BA0994303132333435363738393031D7
:101FA000A5BAED91A5BAFE2FFF73A5BAE078E0655A
:101FB000A5BA0994303132333435363738393031B7
:101FC000A5BAED91A5BAFE2FFF73A5BAE078E06639
:101FD000A5BA099430313233343536373839303197
:101FE000A5BAED91A5BAFE2FFF73A5BAE078E06718
:101FF000A5BA099430313233343536373839303177
:1020000095BAED9195BAFE2FFF7395BAE078E0602E
:1020100095BA099430313233343536373839303166
:1020200095BAED9195BAFE2FFF7395BAE078E0610D
:1020300095BA099430313233343536373839303146
:1020400095BAED9195BAFE2FFF7395BAE078E062EC
:1020500095BA099430313233343536373839303126
:1020600095BAED9195BAFE2FFF7395BAE078E063CB
:1020700095BA099430313233343536373839303106
:1020800095BAED9195BAFE2FFF7395BAE078E064AA
:1020900095BA0994303132333435363738393031E6
:1020A00095BAED9195BAFE2FFF7395BAE078E06589
:1020B00095BA0994303132333435363738393031C6
:1020C00095BAED9195BAFE2FFF7395BAE078E06668
:1020D00095BA0994303132333435363738393031A6
:1020E00095BAED9195BAFE2FFF7395BAE078E06747
:1020F00095BA099430313233343536373839303186
:1021000095BAED9195BAFE2FFF7395BAE078E0602D
:1021100095BA099430313233343536373839303165
:1021200095BAED91A5BAFE2FFF7395BAE078E061FC
:1021300095BA099430313233343536373839303145
:1021400095BAED91A5BAFE2FFF7395BAE078E062DB
:1021500095BA099430313233343536373839303125
:1021600095BAED91A5BAFE2FFF7395BAE078E063BA
:1021700095BA099430313233343536373839303105
:1021800095BAED91A5BAFE2FFF7395BAE078E06499
:1021900095BA0994303132333435363738393031E5
:1021A00095BAED9195BAFE2FFF7395BAE078E06588
:1021B00095BA0994303132333435363738393031C5
:1021C00095BAED91A5BAFE2FFF7395BAE078E06657
:1021D00095BA0994303132333435363738393031A5
:1021E00095BAED9195BAFE2FFF7395BAE078E06746
:1021F00095BA099430313233343536373839303185
:1022000095BAED9195BAFE2FFF7395BAE078E0602C
:1022100095BA099430313233343536373839303164
:10222000A5BAED9195BAFE2FFF73A5BAE078E061EB
:1022300095BA099430313233343536373839303144
:10224000A5BAED9195BAFE2FFF73A5BAE078E062CA
:1022500095BA099430313233343536373839303124
:1022600095BAED9195BAFE2FFF7395BAE078E063C9
:1022700095BA099430313233343536373839303104
:1022800095BAED9195BAFE2FFF7395BAE078E064A8
:1022900095BA0994303132333435363738393031E4
:1022A00095BAED9195BAFE2FFF7395BAE078E06587
:1022B00095BA0994303132333435363738393031C4
:1022C00095BAED9195BAFE2FFF7395BAE078E06666
:1022D00095BA0994303132333435363738393031A4
:1022E00095BAED9195BAFE2FFF7395BAE078E06745
:1022F00095BA099430313233343536373839303184
:1023000095BAED9195BAFE2FFF7395BAE078E0602B
:1023100095BA099430313233343536373839303163
:10232000A5BAED9195BAFE2FFF73A5BAE078E061EA
:1023300095BA099430313233343536373839303143
:10234000A5BAED9195BAFE2FFF73A5BAE078E062C9
:1023500095BA099430313233343536373839303123
:10236000A5BAED91A5BAFE2FFF73A5BAE078E06398
:1023700095BA099430313233343536373839303103
:10238000A5BAED9195BAFE2FFF73A5BAE078E06487
:1023900095BA0994303132333435363738393031E3
:1023A000A5BAED91A5BAFE2FFF73A5BAE078E06556
:1023B00095BA0994303132333435363738393031C3
:1023C000A5BAED9195BAFE2FFF73A5BAE078E06645
:1023D00095BA0994303132333435363738393031A3
:1023E000A5BAED9195BAFE2FFF73A5BAE078E06724
:1023F00095BA099430313233343536373839303183
:1024000095BAED9195BAFE2FFF7395BAE078E0602A
:1024100095BA099430313233343536373839303162
:1024200095BAED91A5BAFE2FFF7395BAE078E061F9
:1024300095BA099430313233343536373839303142
:1024400095BAED91A5BAFE2FFF73A5BAE078E062C8
:1024500095BA099430313233343536373839303122
:10246000A5BAED91A5BAFE2FFF7395BAE078E063A7
:1024700095BA099430313233343536373839303102
:1024800095BAED91A5BAFE2FFF7395BAE078E06496
:1024900095BA0994303132333435363738393031E2
:1024A00095BAED91A5BAFE2FFF73A5BAE078E06565
:1024B00095BA0994303132333435363738393031C2
:1024C000A5BAED91A5BAFE2FFF7395BAE078E06644
:1024D00095BA0994303132333435363738393031A2
:1024E00095BAED91A5BAFE2FFF7395BAE078E06733
:1024F00095BA099430313233343536373839303182
:1025000095BAED9195BAFE2FFF7395BAE078E06029
:1025100095BA099430313233343536373839303161
:10252000A5BAED9195BAFE2FFF73A5BAE078E061E8
:1025300095BA099430313233343536373839303141
:1025400095BAED9195BAFE2FFF73A5BAE078E062D7
:1025500095BA099430313233343536373839303121
:1025600095BAED91A5BAFE2FFF7395BAE078E063B6
:1025700095BA099430313233343536373839303101
:1025800095BAED91A5BAFE2FFF7395BAE078E06495
:1025900095BA0994303132333435363738393031E1
:1025A000A5BAED9195BAFE2FFF7395BAE078E06574
:1025B00095BA0994303132333435363738393031C1
:1025C000A5BAED9195BAFE2FFF73A5BAE078E06643
:1025D00095BA0994303132333435363738393031A1
:1025E00095BAED9195BAFE2FFF7395BAE078E06742
:1025F00095BA099430313233343536373839303181
:1026000095BAED9195BAFE2FFF7395BAE078E06028
:1026100095BA099430313233343536373839303160
:1026200095BAED91A5BAFE2FFF7395BAE078E061F7
:1026300095BA099430313233343536373839303140
:10264000A5BAED9195BAFE2FFF73A5BAE078E062C6
:1026500095BA099430313233343536373839303120
:1026600095BAED91A5BAFE2FFF7395BAE078E063B5
:1026700095BA099430313233343536373839303100
:10268000A5BAED9195BAFE2FFF73A5BAE078E06484
:1026900095BA0994303132333435363738393031E0
:1026A000A5BAED9195BAFE2FFF73A5BAE078E06563
:1026B00095BA0994303132333435363738393031C0
:1026C00095BAED91A5BAFE2FFF73A5BAE078E06642
:1026D00095BA0994303132333435363738393031A0
:1026E00095BAED9195BAFE2FFF7395BAE078E06741
:1026F00095BA099430313233343536373839303180
:1027000095BAED9195BAFE2FFF7395BAE078E06027
:1027100095BA09943031323334353637383930315F
:1027200095BAED91A5BAFE2FFF7395BAE078E061F6
:1027300095BA09943031323334353637383930313F
:10274000A5BAED9195BAFE2FFF7395BAE078E062D5
:1027500095BA09943031323334353637383930311F
:1027600095BAED9195BAFE2FFF7395BAE078E063C4
:1027700095BA0994303132333435363738393031FF
:1027800095BAED9195BAFE2FFF7395BAE078E064A3
:1027900095BA0994303132333435363738393031DF
:1027A00095BAED9195BAFE2FFF7395BAE078E06582
:1027B00095BA0994303132333435363738393031BF
:1027C00095BAED9195BAFE2FFF7395BAE078E06661
:1027D00095BA09943031323334353637383930319F
:1027E00095BAED9195BAFE2FFF7395BAE078E06740
:1027F00095BA09943031323334353637383930317F
:1028000095BAED9195BAFE2FFF7395BAE078E06026
:1028100095BA09943031323334353637383930315E
:1028200095BAED91A5BAFE2FFF7395BAE078E061F5
:1028300095BA09943031323334353637383930313E
:10284000A5BAED9195BAFE2FFF7395BAE078E062D4
:1028500095BA09943031323334353637383930311E
:10286000A5BAED9195BAFE2FFF7395BAE078E063B3
:1028700095BA0994303132333435363738393031FE
:10288000A5BAED9195BAFE2FFF7395BAE078E06492
:1028900095BA0994303132333435363738393031DE
:1028A000A5BAED9195BAFE2FFF7395BAE078E06571
:1028B00095BA0994303132333435363738393031BE
:1028C00095BAED91A5BAFE2FFF7395BAE078E06650
:1028D00095BA09943031323334353637383930319E
:1028E00095BAED9195BAFE2FFF7395BAE078E0673F
:1028F00095BA09943031323334353637383930317E
:1029000095BAED9195BAFE2FFF7395BAE078E06025
:1029100095BA09943031323334353637383930315D
:1029200095BAED91A5BAFE2FFF7395BAE078E061F4
:1029300095BA09943031323334353637383930313D
:1029400095BAED9195BAFE2FFF73A5BAE078E062D3
:1029500095BA09943031323334353637383930311D
:1029600095BAED9195BAFE2FFF73A5BAE078E063B2
:1029700095BA0994303132333435363738393031FD
:1029800095BAED9195BAFE2FFF73A5BAE078E06491
:1029900095BA0994303132333435363738393031DD
:1029A00095BAED9195BAFE2FFF73A5BAE078E06570
:1029B00095BA0994303132333435363738393031BD
:1029C00095BAED91A5BAFE2FFF7395BAE078E0664F
:1029D00095BA09943031323334353637383930319D
:1029E00095BAED9195BAFE2FFF7395BAE078E0673E
:1029F00095BA09943031323334353637383930317D
:102A000095BAED9195BAFE2FFF7395BAE078E06024
:102A100095BA09943031323334353637383930315C
:102A200095BAED9195BAFE2FFF7395BAE078E06103
:102A300095BA09943031323334353637383930313C
:102A400095BAED91A5BAFE2FFF7395BAE078E062D2
:102A500095BA09943031323334353637383930311C
:102A6000A5BAED91A5BAFE2FFF73A5BAE078E06391
:102A700095BA0994303132333435363738393031FC
:102A800095BAED91A5BAFE2FFF7395BAE078E06490
:102A900095BA0994303132333435363738393031DC
:102AA000A5BAED91A5BAFE2FFF73A5BAE078E0654F
:102AB00095BA0994303132333435363738393031BC
:102AC00095BAED91A5BAFE2FFF7395BAE078E0664E
:102AD00095BA09943031323334353637383930319C
:102AE00095BAED9195BAFE2FFF7395BAE078E0673D
:102AF00095BA09943031323334353637383930317C
:102B000095BAED9195BAFE2FFF7395BAE078E06023
:102B100095BA09943031323334353637383930315B
:102B200095BAED9195BAFE2FFF7395BAE078E06102
:102B300095BA09943031323334353637383930313B
:102B400095BAED91A5BAFE2FFF7395BAE078E062D1
:102B500095BA09943031323334353637383930311B
:102B600095BAED91A5BAFE2FFF7395BAE078E063B0
:102B700095BA0994303132333435363738393031FB
:102B8000A5BAED91A5BAFE2FFF73A5BAE078E0646F
:102B900095BA0994303132333435363738393031DB
:102BA00095BAED91A5BAFE2FFF7395BAE078E0656E
:102BB00095BA0994303132333435363738393031BB
:102BC00095BAED91A5BAFE2FFF7395BAE078E0664D
:102BD00095BA09943031323334353637383930319B
:102BE00095BAED9195BAFE2FFF7395BAE078E0673C
:102BF00095BA09943031323334353637383930317B
:102C000095BAED9195BAFE2FFF7395BAE078E06022
:102C100095BA09943031323334353637383930315A
:102C200095BAED9195BAFE2FFF7395BAE078E06101
:102C300095BA09943031323334353637383930313A
:102C400095BAED9195BAFE2FFF7395BAE078E062E0
:102C500095BA09943031323334353637383930311A
:102C600095BAED9195BAFE2FFF7395BAE078E063BF
:102C700095BA0994303132333435363738393031FA
:102C800095BAED9195BAFE2FFF7395BAE078E0649E
:102C900095BA0994303132333435363738393031DA
:102CA00095BAED91A5BAFE2FFF7395BAE078E0656D
:102CB00095BA0994303132333435363738393031BA
:102CC00095BAED91A5BAFE2FFF7395BAE078E0664C
:102CD00095BA09943031323334353637383930319A
:102CE000A5BAED9195BAFE2FFF7395BAE078E0672B
:102CF00095BA09943031323334353637383930317A
:102D000095BAED9195BAFE2FFF7395BAE078E06021
:102D100095BA099430313233343536373839303159
:102D200095BAED9195BAFE2FFF7395BAE078E06100
:102D300095BA099430313233343536373839303139
:102D400095BAED9195BAFE2FFF7395BAE078E062DF
:102D500095BA099430313233343536373839303119
:102D600095BAED9195BAFE2FFF7395BAE078E063BE
:102D700095BA0994303132333435363738393031F9
:102D8000A5BAED91A5BAFE2FFF73A5BAE078E0646D
:102D900095BA0994303132333435363738393031D9
:102DA00095BAED9195BAFE2FFF7395BAE078E0657C
:102DB00095BA0994303132333435363738393031B9
:102DC00095BAED9195BAFE2FFF7395BAE078E0665B
:102DD00095BA099430313233343536373839303199
:102DE00095BAED9195BAFE2FFF7395BAE078E0673A
:102DF00095BA099430313233343536373839303179
:102E000095BAED9195BAFE2FFF7395BAE078E06020
:102E100095BA099430313233343536373839303158
:102E200095BAED9195BAFE2FFF7395BAE078E061FF
:102E300095BA099430313233343536373839303138
:102E400095BAED9195BAFE2FFF7395BAE078E062DE
:102E500095BA099430313233343536373839303118
:102E600095BAED9195BAFE2FFF7395BAE078E063BD
:102E700095BA0994303132333435363738393031F8
:102E800095BAED9195BAFE2FFF7395BAE078E0649C
:102E900095BA0994303132333435363738393031D8
:102EA00095BAED91A5BAFE2FFF7395BAE078E0656B
:102EB00095BA0994303132333435363738393031B8
:102EC00095BAED91A5BAFE2FFF7395BAE078E0664A
:102ED00095BA099430313233343536373839303198
:102EE00095BAED9195BAFE2FFF7395BAE078E06739
:102EF00095BA099430313233343536373839303178
:102F000095BAED9195BAFE2FFF7395BAE078E0601F
:102F100095BA099430313233343536373839303157
:102F200095BAED9195BAFE2FFF73A5BAE078E061EE
:102F300095BA099430313233343536373839303137
:102F400095BAED9195BAFE2FFF73A5BAE078E062CD
:102F500095BA099430313233343536373839303117
:102F600095BAED91A5BAFE2FFF7395BAE078E063AC
:102F700095BA0994303132333435363738393031F7
:102F800095BAED91A5BAFE2FFF7395BAE078E0648B
:102F900095BA0994303132333435363738393031D7
:102FA000A5BAED9195BAFE2FFF7395BAE078E0656A
:102FB00095BA0994303132333435363738393031B7
:102FC000A5BAED9195BAFE2FFF7395BAE078E06649
:102FD00095BA099430313233343536373839303197
:102FE00095BAED9195BAFE2FFF7395BAE078E06738
:102FF00095BA099430313233343536373839303177
:1030000095BAED9195BAFE2FFF7395BAE078E0601E
:1030100095BA099430313233343536373839303156
:1030200095BAED91A5BAFE2FFF7395BAE078E061ED
:1030300095BA099430313233343536373839303136
:10304000A5BAED9195BAFE2FFF73A5BAE078E062BC
:1030500095BA099430313233343536373839303116
:10306000A5BAED9195BAFE2FFF73A5BAE078E0639B
:1030700095BA0994303132333435363738393031F6
:10308000A5BAED9195BAFE2FFF73A5BAE078E0647A
:1030900095BA0994303132333435363738393031D6
:1030A000A5BAED9195BAFE2FFF73A5BAE078E06559
:1030B00095BA0994303132333435363738393031B6
:1030C00095BAED91A5BAFE2FFF7395BAE078E06648
:1030D00095BA099430313233343536373839303196
:1030E00095BAED9195BAFE2FFF7395BAE078E06737
:1030F00095BA099430313233343536373839303176
:1031000095BAED9195BAFE2FFF7395BAE078E0601D
:1031100095BA099430313233343536373839303155
:1031200095BAED91A5BAFE2FFF7395BAE078E061EC
:1031300095BA099430313233343536373839303135
:10314000A5BAED91A5BAFE2FFF7395BAE078E062BB
:1031500095BA099430313233343536373839303115
:1031600095BAED91A5BAFE2FFF7395BAE078E063AA
:1031700095BA0994303132333435363738393031F5
:1031800095BAED91A5BAFE2FFF7395BAE078E06489
:1031900095BA0994303132333435363738393031D5
:1031A00095BAED91A5BAFE2FFF7395BAE078E06568
:1031B00095BA0994303132333435363738393031B5
:1031C000A5BAED91A5BAFE2FFF73A5BAE078E06627
:1031D00095BA099430313233343536373839303195
:1031E00095BAED9195BAFE2FFF7395BAE078E06736
:1031F00095BA099430313233343536373839303175
:1032000095BAED9195BAFE2FFF7395BAE078E0601C
:1032100095BA099430313233343536373839303154
:10322000A5BAED91A5BAFE2FFF7395BAE078E061DB
:1032300095BA099430313233343536373839303134
:1032400095BAED9195BAFE2FFF73A5BAE078E062CA
:1032500095BA099430313233343536373839303114
:1032600095BAED9195BAFE2FFF73A5BAE078E063A9
:1032700095BA0994303132333435363738393031F4
:1032800095BAED91A5BAFE2FFF7395BAE078E06488
:1032900095BA0994303132333435363738393031D4
:1032A000A5BAED9195BAFE2FFF7395BAE078E06567
:1032B00095BA0994303132333435363738393031B4
:1032C000A5BAED91A5BAFE2FFF73A5BAE078E06626
:1032D00095BA099430313233343536373839303194
:1032E00095BAED9195BAFE2FFF7395BAE078E06735
:1032F00095BA099430313233343536373839303174
:1033000095BAED9195BAFE2FFF7395BAE078E0601B
:1033100095BA099430313233343536373839303153
:10332000A5BAED91A5BAFE2FFF7395BAE078E061DA
:1033300095BA099430313233343536373839303133
:1033400095BAED9195BAFE2FFF73A5BAE078E062C9
:1033500095BA099430313233343536373839303113
:1033600095BAED91A5BAFE2FFF7395BAE078E063A8
:1033700095BA0994303132333435363738393031F3
:1033800095BAED9195BAFE2FFF73A5BAE078E06487
:1033900095BA0994303132333435363738393031D3
:1033A00095BAED9195BAFE2FFF73A5BAE078E06566
:1033B00095BA0994303132333435363738393031B3
:1033C000A5BAED91A5BAFE2FFF7395BAE078E06635
:1033D00095BA099430313233343536373839303193
:1033E00095BAED9195BAFE2FFF7395BAE078E06734
:1033F00095BA099430313233343536373839303173
:1034000095BAED9195BAFE2FFF7395BAE078E0601A
:1034100095BA099430313233343536373839303152
:10342000A5BAED9195BAFE2FFF7395BAE078E061E9
:1034300095BA099430313233343536373839303132
:10344000A5BAED9195BAFE2FFF73A5BAE078E062B8
:1034500095BA099430313233343536373839303112
:10346000A5BAED9195BAFE2FFF73A5BAE078E06397
:1034700095BA0994303132333435363738393031F2
:10348000A5BAED91A5BAFE2FFF73A5BAE078E06466
:1034900095BA0994303132333435363738393031D2
:1034A00095BAED9195BAFE2FFF73A5BAE078E06565
:1034B00095BA0994303132333435363738393031B2
:1034C00095BAED9195BAFE2FFF73A5BAE078E06644
:1034D00095BA099430313233343536373839303192
:1034E00095BAED9195BAFE2FFF7395BAE078E06733
:1034F00095BA099430313233343536373839303172
:1035000095BAED9195BAFE2FFF7395BAE078E06019
:1035100095BA099430313233343536373839303151
:10352000A5BAED91A5BAFE2FFF73A5BAE078E061C8
:1035300095BA099430313233343536373839303131
:10354000A5BAED9195BAFE2FFF7395BAE078E062C7
:1035500095BA099430313233343536373839303111
:10356000A5BAED91A5BAFE2FFF7395BAE078E06396
:1035700095BA0994303132333435363738393031F1
:1035800095BAED9195BAFE2FFF73A5BAE078E06485
:1035900095BA0994303132333435363738393031D1
:1035A00095BAED9195BAFE2FFF73A5BAE078E06564
:1035B00095BA0994303132333435363738393031B1
:1035C000A5BAED91A5BAFE2FFF7395BAE078E06633
:1035D00095BA099430313233343536373839303191
:1035E00095BAED9195BAFE2FFF7395BAE078E06732
:1035F00095BA099430313233343536373839303171
:1036000095BAED9195BAFE2FFF7395BAE078E06018
:1036100095BA099430313233343536373839303150
:1036200095BAED91A5BAFE2FFF7395BAE078E061E7
:1036300095BA099430313233343536373839303130
:10364000A5BAED9195BAFE2FFF7395BAE078E062C6
:1036500095BA099430313233343536373839303110
:10366000A5BAED91A5BAFE2FFF7395BAE078E06395
:1036700095BA0994303132333435363738393031F0
:10368000A5BAED9195BAFE2FFF73A5BAE078E06474
:1036900095BA0994303132333435363738393031D0
:1036A000A5BAED9195BAFE2FFF73A5BAE078E06553
:1036B00095BA0994303132333435363738393031B0
:1036C00095BAED91A5BAFE2FFF7395BAE078E06642
:1036D00095BA099430313233343536373839303190
:1036E00095BAED9195BAFE2FFF7395BAE078E06731
:1036F00095BA099430313233343536373839303170
:1037000095BAED9195BAFE2FFF7395BAE078E06017
:1037100095BA09943031323334353637383930314F
:10372000A5BAED91A5BAFE2FFF73A5BAE078E061C6
:1037300095BA09943031323334353637383930312F
:1037400095BAED9195BAFE2FFF73A5BAE078E062C5
:1037500095BA09943031323334353637383930310F
:1037600095BAED9195BAFE2FFF73A5BAE078E063A4
:1037700095BA0994303132333435363738393031EF
:1037800095BAED91A5BAFE2FFF7395BAE078E06483
:1037900095BA0994303132333435363738393031CF
:1037A000A5BAED9195BAFE2FFF7395BAE078E06562
:1037B00095BA0994303132333435363738393031AF
:1037C000A5BAED9195BAFE2FFF7395BAE078E06641
:1037D00095BA09943031323334353637383930318F
:1037E00095BAED9195BAFE2FFF7395BAE078E06730
:1037F00095BA09943031323334353637383930316F
:1038000095BAED9195BAFE2FFF7395BAE078E06016
:1038100095BA09943031323334353637383930314E
:1038200095BAED91A5BAFE2FFF7395BAE078E061E5
:1038300095BA09943031323334353637383930312E
:10384000A5BAED9195BAFE2FFF73A5BAE078E062B4
:1038500095BA09943031323334353637383930310E
:1038600095BAED91A5BAFE2FFF7395BAE078E063A3
:1038700095BA0994303132333435363738393031EE
:10388000A5BAED9195BAFE2FFF73A5BAE078E06472
:1038900095BA0994303132333435363738393031CE
:1038A000A5BAED9195BAFE2FFF73A5BAE078E06551
:1038B00095BA0994303132333435363738393031AE
:1038C00095BAED91A5BAFE2FFF7395BAE078E06640
:1038D00095BA09943031323334353637383930318E
:1038E00095BAED9195BAFE2FFF7395BAE078E0672F
:1038F00095BA09943031323334353637383930316E
:1039000095BAED9195BAFE2FFF7395BAE078E06015
:1039100095BA09943031323334353637383930314D
:1039200095BAED91A5BAFE2FFF7395BAE078E061E4
:1039300095BA09943031323334353637383930312D
:10394000A5BAED9195BAFE2FFF73A5BAE078E062B3
:1039500095BA09943031323334353637383930310D
:10396000A5BAED9195BAFE2FFF73A5BAE078E06392
:1039700095BA0994303132333435363738393031ED
:1039800095BAED91A5BAFE2FFF73A5BAE078E06471
:1039900095BA0994303132333435363738393031CD
:1039A00095BAED9195BAFE2FFF73A5BAE078E06560
:1039B00095BA0994303132333435363738393031AD
:1039C00095BAED91A5BAFE2FFF7395BAE078E0663F
:1039D00095BA09943031323334353637383930318D
:1039E00095BAED9195BAFE2FFF7395BAE078E0672E
:1039F00095BA09943031323334353637383930316D
:103A000095BAED9195BAFE2FFF7395BAE078E06014
:103A100095BA09943031323334353637383930314C
:103A200095BAED9195BAFE2FFF7395BAE078E061F3
:103A300095BA09943031323334353637383930312C
:103A400095BAED91A5BAFE2FFF7395BAE078E062C2
:103A500095BA09943031323334353637383930310C
:103A600095BAED91A5BAFE2FFF7395BAE078E063A1
:103A700095BA0994303132333435363738393031EC
:103A800095BAED9195BAFE2FFF7395BAE078E06490
:103A900095BA0994303132333435363738393031CC
:103AA00095BAED91A5BAFE2FFF7395BAE078E0655F
:103AB00095BA0994303132333435363738393031AC
:103AC00095BAED91A5BAFE2FFF7395BAE078E0663E
:103AD00095BA09943031323334353637383930318C
:103AE00095BAED9195BAFE2FFF7395BAE078E0672D
:103AF00095BA09943031323334353637383930316C
:103B000095BAED9195BAFE2FFF7395BAE078E06013
:103B100095BA09943031323334353637383930314B
:103B200095BAED9195BAFE2FFF7395BAE078E061F2
:103B300095BA09943031323334353637383930312B
:103B400095BAED91A5BAFE2FFF7395BAE078E062C1
:103B500095BA09943031323334353637383930310B
:103B600095BAED91A5BAFE2FFF7395BAE078E063A0
:103B700095BA0994303132333435363738393031EB
:103B800095BAED9195BAFE2FFF7395BAE078E0648F
:103B900095BA0994303132333435363738393031CB
:103BA00095BAED91A5BAFE2FFF7395BAE078E0655E
:103BB00095BA0994303132333435363738393031AB
:103BC00095BAED91A5BAFE2FFF7395BAE078E0663D
:103BD00095BA09943031323334353637383930318B
:103BE000A5BAED9195BAFE2FFF7395BAE078E0671C
:103BF00095BA09943031323334353637383930316B
:103C000095BAED9195BAFE2FFF7395BAE078E06012
:103C100095BA09943031323334353637383930314A
:103C200095BAED9195BAFE2FFF7395BAE078E061F1
:103C300095BA09943031323334353637383930312A
:103C400095BAED9195BAFE2FFF73A5BAE078E062C0
:103C500095BA09943031323334353637383930310A
:103C600095BAED91A5BAFE2FFF7395BAE078E0639F
:103C700095BA0994303132333435363738393031EA
:103C8000A5BAED9195BAFE2FFF7395BAE078E0647E
:103C900095BA0994303132333435363738393031CA
:103CA00095BAED91A5BAFE2FFF7395BAE078E0655D
:103CB00095BA0994303132333435363738393031AA
:103CC00095BAED9195BAFE2FFF73A5BAE078E0663C
:103CD00095BA09943031323334353637383930318A
:103CE00095BAED9195BAFE2FFF7395BAE078E0672B
:103CF00095BA09943031323334353637383930316A
:103D000095BAED9195BAFE2FFF7395BAE078E06011
:103D100095BA099430313233343536373839303149
:103D200095BAED9195BAFE2FFF7395BAE078E061F0
:103D300095BA099430313233343536373839303129
:103D400095BAED9195BAFE2FFF7395BAE078E062CF
:103D500095BA099430313233343536373839303109
:103D6000A5BAED91A5BAFE2FFF73A5BAE078E0637E
:103D700095BA0994303132333435363738393031E9
:103D800095BAED9195BAFE2FFF7395BAE078E0648D
:103D900095BA0994303132333435363738393031C9
:103DA000A5BAED91A5BAFE2FFF73A5BAE078E0653C
:103DB00095BA0994303132333435363738393031A9
:103DC00095BAED9195BAFE2FFF7395BAE078E0664B
:103DD00095BA099430313233343536373839303189
:103DE00095BAED9195BAFE2FFF7395BAE078E0672A
:103DF00095BA099430313233343536373839303169
:103E000095BAED9195BAFE2FFF7395BAE078E06010
:103E100095BA099430313233343536373839303148
:103E200095BAED9195BAFE2FFF7395BAE078E061EF
:103E300095BA099430313233343536373839303128
:103E4000A5BAED9195BAFE2FFF7395BAE078E062BE
:103E500095BA099430313233343536373839303108
:103E600095BAED91A5BAFE2FFF7395BAE078E0639D
:103E700095BA0994303132333435363738393031E8
:103E800095BAED9195BAFE2FFF73A5BAE078E0647C
:103E900095BA0994303132333435363738393031C8
:103EA00095BAED91A5BAFE2FFF7395BAE078E0655B
:103EB00095BA0994303132333435363738393031A8
:103EC000A5BAED9195BAFE2FFF7395BAE078E0663A
:103ED00095BA099430313233343536373839303188
:103EE00095BAED9195BAFE2FFF7395BAE078E06729
:103EF00095BA099430313233343536373839303168
:103F000095BAED9195BAFE2FFF7395BAE078E0600F
:103F100095BA099430313233343536373839303147
:103F2000A5BAED91A5BAFE2FFF7395BAE078E061CE
:103F300095BA099430313233343536373839303127
:103F400095BAED9195BAFE2FFF73A5BAE078E062BD
:103F500095BA099430313233343536373839303107
:103F600095BAED91A5BAFE2FFF7395BAE078E0639C
:103F700095BA0994303132333435363738393031E7
:103F800095BAED91A5BAFE2FFF7395BAE078E0647B
:103F900095BA0994303132333435363738393031C7
:103FA00095BAED9195BAFE2FFF7395BAE078E0656A
:103FB00095BA0994303132333435363738393031A7
:103FC00095BAED91A5BAFE2FFF7395BAE078E06639
:103FD00095BA099430313233343536373839303187
:103FE00095BAED9195BAFE2FFF7395BAE078E06728
:103FF00095BA099430313233343536373839303167
:1040000095BAED9195BAFE2FFF7395BAE078E0600E
:1040100095BA099430313233343536373839303146
:1040200095BAED91A5BAFE2FFF7395BAE078E061DD
:1040300095BA099430313233343536373839303126
:10404000A5BAED9195BAFE2FFF73A5BAE078E062AC
:1040500095BA099430313233343536373839303106
:10406000A5BAED91A5BAFE2FFF73A5BAE078E0637B
:1040700095BA0994303132333435363738393031E6
:10408000A5BAED91A5BAFE2FFF73A5BAE078E0645A
:1040900095BA0994303132333435363738393031C6
:1040A000A5BAED9195BAFE2FFF7395BAE078E06559
:1040B00095BA0994303132333435363738393031A6
:1040C00095BAED91A5BAFE2FFF73A5BAE078E06628
:1040D00095BA099430313233343536373839303186
:1040E00095BAED9195BAFE2FFF7395BAE078E06727
:1040F00095BA099430313233343536373839303166
:1041000095BAED9195BAFE2FFF7395BAE078E0600D
:1041100095BA099430313233343536373839303145
:1041200095BAED91A5BAFE2FFF7395BAE078E061DC
:1041300095BA099430313233343536373839303125
:10414000A5BAED9195BAFE2FFF73A5BAE078E062AB
:1041500095BA099430313233343536373839303105
:10416000A5BAED9195BAFE2FFF73A5BAE078E0638A
:1041700095BA0994303132333435363738393031E5
:10418000A5BAED91A5BAFE2FFF73A5BAE078E06459
:1041900095BA0994303132333435363738393031C5
:1041A000A5BAED9195BAFE2FFF73A5BAE078E06548
:1041B00095BA0994303132333435363738393031A5
:1041C000A5BAED9195BAFE2FFF73A5BAE078E06627
:1041D00095BA099430313233343536373839303185
:1041E00095BAED9195BAFE2FFF7395BAE078E06726
:1041F00095BA099430313233343536373839303165
:1042000095BAED9195BAFE2FFF7395BAE078E0600C
:1042100095BA099430313233343536373839303144
:10422000A5BAED91A5BAFE2FFF7395BAE078E061CB
:1042300095BA099430313233343536373839303124
:10424000A5BAED9195BAFE2FFF73A5BAE078E062AA
:1042500095BA099430313233343536373839303104
:10426000A5BAED91A5BAFE2FFF7395BAE078E06389
:1042700095BA0994303132333435363738393031E4
:10428000A5BAED9195BAFE2FFF73A5BAE078E06468
:1042900095BA0994303132333435363738393031C4
:1042A000A5BAED9195BAFE2FFF73A5BAE078E06547
:1042B00095BA0994303132333435363738393031A4
:1042C000A5BAED91A5BAFE2FFF7395BAE078E06626
:1042D00095BA099430313233343536373839303184
:1042E00095BAED9195BAFE2FFF7395BAE078E06725
:1042F00095BA099430313233343536373839303164
:1043000095BAED9195BAFE2FFF7395BAE078E0600B
:1043100095BA099430313233343536373839303143
:1043200095BAED91A5BAFE2FFF73A5BAE078E061CA
:1043300095BA099430313233343536373839303123
:10434000A5BAED9195BAFE2FFF7395BAE078E062B9
:1043500095BA099430313233343536373839303103
:10436000A5BAED9195BAFE2FFF7395BAE078E06398
:1043700095BA0994303132333435363738393031E3
:10438000A5BAED9195BAFE2FFF7395BAE078E06477
:1043900095BA0994303132333435363738393031C3
:1043A000A5BAED9195BAFE2FFF7395BAE078E06556
:1043B00095BA0994303132333435363738393031A3
:1043C00095BAED91A5BAFE2FFF73A5BAE078E06625
:1043D00095BA099430313233343536373839303183
:1043E00095BAED9195BAFE2FFF7395BAE078E06724
:1043F00095BA099430313233343536373839303163
:1044000095BAED9195BAFE2FFF7395BAE078E0600A
:1044100095BA099430313233343536373839303142
:10442000A5BAED91A5BAFE2FFF7395BAE078E061C9
:1044300095BA099430313233343536373839303122
:10444000A5BAED9195BAFE2FFF73A5BAE078E062A8
:1044500095BA099430313233343536373839303102
:10446000A5BAED9195BAFE2FFF73A5BAE078E06387
:1044700095BA0994303132333435363738393031E2
:10448000A5BAED9195BAFE2FFF73A5BAE078E06466
:1044900095BA0994303132333435363738393031C2
:1044A000A5BAED9195BAFE2FFF73A5BAE078E06545
:1044B00095BA0994303132333435363738393031A2
:1044C000A5BAED91A5BAFE2FFF7395BAE078E06624
:1044D00095BA099430313233343536373839303182
:1044E00095BAED9195BAFE2FFF7395BAE078E06723
:1044F00095BA099430313233343536373839303162
:1045000095BAED9195BAFE2FFF7395BAE078E06009
:1045100095BA099430313233343536373839303141
:10452000A5BAED91A5BAFE2FFF73A5BAE078E061B8
:1045300095BA099430313233343536373839303121
:10454000A5BAED9195BAFE2FFF7395BAE078E062B7
:1045500095BA099430313233343536373839303101
:10456000A5BAED91A5BAFE2FFF7395BAE078E06386
:1045700095BA0994303132333435363738393031E1
:10458000A5BAED9195BAFE2FFF7395BAE078E06475
:1045900095BA0994303132333435363738393031C1
:1045A000A5BAED9195BAFE2FFF7395BAE078E06554
:1045B00095BA0994303132333435363738393031A1
:1045C000A5BAED91A5BAFE2FFF73A5BAE078E06613
:1045D00095BA099430313233343536373839303181
:1045E00095BAED9195BAFE2FFF7395BAE078E06722
:1045F00095BA099430313233343536373839303161
:1046000095BAED9195BAFE2FFF7395BAE078E06008
:1046100095BA099430313233343536373839303140
:10462000A5BAED91A5BAFE2FFF73A5BAE078E061B7
:1046300095BA099430313233343536373839303120
:10464000A5BAED9195BAFE2FFF7395BAE078E062B6
:1046500095BA099430313233343536373839303100
:10466000A5BAED9195BAFE2FFF7395BAE078E06395
:1046700095BA0994303132333435363738393031E0
:10468000A5BAED91A5BAFE2FFF7395BAE078E06464
:1046900095BA0994303132333435363738393031C0
:1046A000A5BAED9195BAFE2FFF7395BAE078E06553
:1046B00095BA0994303132333435363738393031A0
:1046C000A5BAED9195BAFE2FFF7395BAE078E06632
:1046D00095BA099430313233343536373839303180
:1046E00095BAED9195BAFE2FFF7395BAE078E06721
:1046F00095BA099430313233343536373839303160
:1047000095BAED9195BAFE2FFF7395BAE078E06007
:1047100095BA09943031323334353637383930313F
:1047200095BAED91A5BAFE2FFF73A5BAE078E061C6
:1047300095BA09943031323334353637383930311F
:10474000A5BAED9195BAFE2FFF7395BAE078E062B5
:1047500095BA0994303132333435363738393031FF
:10476000A5BAED9195BAFE2FFF7395BAE078E06394
:1047700095BA0994303132333435363738393031DF
:10478000A5BAED9195BAFE2FFF73A5BAE078E06463
:1047900095BA0994303132333435363738393031BF
:1047A000A5BAED9195BAFE2FFF73A5BAE078E06542
:1047B00095BA09943031323334353637383930319F
:1047C00095BAED91A5BAFE2FFF73A5BAE078E06621
:1047D00095BA09943031323334353637383930317F
:1047E00095BAED9195BAFE2FFF7395BAE078E06720
:1047F00095BA09943031323334353637383930315F
:1048000095BAED9195BAFE2FFF7395BAE078E06006
:1048100095BA09943031323334353637383930313E
:10482000A5BAED9195BAFE2FFF73A5BAE078E061C5
:1048300095BA09943031323334353637383930311E
:10484000A5BAED9195BAFE2FFF73A5BAE078E062A4
:1048500095BA0994303132333435363738393031FE
:10486000A5BAED91A5BAFE2FFF73A5BAE078E06373
:1048700095BA0994303132333435363738393031DE
:10488000A5BAED9195BAFE2FFF73A5BAE078E06462
:1048900095BA0994303132333435363738393031BE
:1048A000A5BAED9195BAFE2FFF73A5BAE078E06541
:1048B00095BA09943031323334353637383930319E
:1048C000A5BAED9195BAFE2FFF73A5BAE078E06620
:1048D00095BA09943031323334353637383930317E
:1048E00095BAED9195BAFE2FFF7395BAE078E0671F
:1048F00095BA09943031323334353637383930315E
:1049000095BAED9195BAFE2FFF7395BAE078E06005
:1049100095BA09943031323334353637383930313D
:10492000A5BAED91A5BAFE2FFF73A5BAE078E061B4
:1049300095BA09943031323334353637383930311D
:1049400095BAED91A5BAFE2FFF7395BAE078E062B3
:1049500095BA0994303132333435363738393031FD
:1049600095BAED91A5BAFE2FFF7395BAE078E06392
:1049700095BA0994303132333435363738393031DD
:1049800095BAED91A5BAFE2FFF7395BAE078E06471
:1049900095BA0994303132333435363738393031BD
:1049A00095BAED91A5BAFE2FFF7395BAE078E06550
:1049B00095BA09943031323334353637383930319D
:1049C000A5BAED91A5BAFE2FFF73A5BAE078E0660F
:1049D00095BA09943031323334353637383930317D
:1049E00095BAED9195BAFE2FFF7395BAE078E0671E
:1049F00095BA09943031323334353637383930315D
:104A000095BAED9195BAFE2FFF7395BAE078E06004
:104A100095BA09943031323334353637383930313C
:104A2000A5BAED91A5BAFE2FFF73A5BAE078E061B3
:104A300095BA09943031323334353637383930311C
:104A400095BAED91A5BAFE2FFF7395BAE078E062B2
:104A500095BA0994303132333435363738393031FC
:104A600095BAED91A5BAFE2FFF7395BAE078E06391
:104A700095BA0994303132333435363738393031DC
:104A800095BAED91A5BAFE2FFF7395BAE078E06470
:104A900095BA0994303132333435363738393031BC
:104AA00095BAED91A5BAFE2FFF7395BAE078E0654F
:104AB00095BA09943031323334353637383930319C
:104AC000A5BAED9195BAFE2FFF7395BAE078E0662E
:104AD00095BA09943031323334353637383930317C
:104AE00095BAED9195BAFE2FFF7395BAE078E0671D
:104AF00095BA09943031323334353637383930315C
:104B000095BAED9195BAFE2FFF7395BAE078E06003
:104B100095BA09943031323334353637383930313B
:104B2000A5BAED9195BAFE2FFF73A5BAE078E061C2
:104B300095BA09943031323334353637383930311B
:104B4000A5BAED9195BAFE2FFF73A5BAE078E062A1
:104B500095BA0994303132333435363738393031FB
:104B6000A5BAED91A5BAFE2FFF7395BAE078E06380
:104B700095BA0994303132333435363738393031DB
:104B8000A5BAED91A5BAFE2FFF7395BAE078E0645F
:104B900095BA0994303132333435363738393031BB
:104BA000A5BAED9195BAFE2FFF73A5BAE078E0653E
:104BB00095BA09943031323334353637383930319B
:104BC000A5BAED9195BAFE2FFF73A5BAE078E0661D
:104BD00095BA09943031323334353637383930317B
:104BE00095BAED9195BAFE2FFF7395BAE078E0671C
:104BF00095BA09943031323334353637383930315B
:104C000095BAED9195BAFE2FFF7395BAE078E06002
:104C100095BA09943031323334353637383930313A
:104C2000A5BAED9195BAFE2FFF7395BAE078E061D1
:104C300095BA09943031323334353637383930311A
:104C4000A5BAED9195BAFE2FFF7395BAE078E062B0
:104C500095BA0994303132333435363738393031FA
:104C6000A5BAED9195BAFE2FFF7395BAE078E0638F
:104C700095BA0994303132333435363738393031DA
:104C8000A5BAED9195BAFE2FFF7395BAE078E0646E
:104C900095BA0994303132333435363738393031BA
:104CA000A5BAED9195BAFE2FFF7395BAE078E0654D
:104CB00095BA09943031323334353637383930319A
:104CC000A5BAED91A5BAFE2FFF73A5BAE078E0660C
:104CD00095BA09943031323334353637383930317A
:104CE00095BAED9195BAFE2FFF7395BAE078E0671B
:104CF00095BA09943031323334353637383930315A
:104D000095BAED9195BAFE2FFF7395BAE078E06001
:104D100095BA099430313233343536373839303139
:104D2000A5BAED9195BAFE2FFF73A5BAE078E061C0
:104D300095BA099430313233343536373839303119
:104D4000A5BAED91A5BAFE2FFF73A5BAE078E0628F
:104D500095BA0994303132333435363738393031F9
:104D6000A5BAED91A5BAFE2FFF73A5BAE078E0636E
:104D700095BA0994303132333435363738393031D9
:104D8000A5BAED9195BAFE2FFF73A5BAE078E0645D
:104D900095BA0994303132333435363738393031B9
:104DA000A5BAED9195BAFE2FFF73A5BAE078E0653C
:104DB00095BA099430313233343536373839303199
:104DC000A5BAED9195BAFE2FFF73A5BAE078E0661B
:104DD00095BA099430313233343536373839303179
:104DE00095BAED9195BAFE2FFF7395BAE078E0671A
:104DF00095BA099430313233343536373839303159
:104E000095BAED9195BAFE2FFF7395BAE078E06000
:104E100095BA099430313233343536373839303138
:104E2000A5BAED9195BAFE2FFF73A5BAE078E061BF
:104E300095BA099430313233343536373839303118
:104E4000A5BAED91A5BAFE2FFF73A5BAE078E0628E
:104E500095BA0994303132333435363738393031F8
:104E6000A5BAED91A5BAFE2FFF73A5BAE078E0636D
:104E700095BA0994303132333435363738393031D8
:104E8000A5BAED91A5BAFE2FFF73A5BAE078E0644C
:104E900095BA0994303132333435363738393031B8
:104EA000A5BAED91A5BAFE2FFF73A5BAE078E0652B
:104EB00095BA099430313233343536373839303198
:104EC000A5BAED9195BAFE2FFF73A5BAE078E0661A
:104ED00095BA099430313233343536373839303178
:104EE00095BAED9195BAFE2FFF7395BAE078E06719
:104EF00095BA099430313233343536373839303158
:104F000095BAED9195BAFE2FFF7395BAE078E060FF
:104F100095BA099430313233343536373839303137
:104F200095BAED91A5BAFE2FFF7395BAE078E061CE
:104F300095BA099430313233343536373839303117
:104F4000A5BAED9195BAFE2FFF73A5BAE078E0629D
:104F500095BA0994303132333435363738393031F7
:104F6000A5BAED9195BAFE2FFF73A5BAE078E0637C
:104F700095BA0994303132333435363738393031D7
:104F8000A5BAED9195BAFE2FFF73A5BAE078E0645B
:104F900095BA0994303132333435363738393031B7
:104FA000A5BAED9195BAFE2FFF73A5BAE078E0653A
:104FB00095BA099430313233343536373839303197
:104FC00095BAED91A5BAFE2FFF7395BAE078E06629
:104FD00095BA099430313233343536373839303177
:104FE00095BAED9195BAFE2FFF7395BAE078E06718
:104FF00095BA099430313233343536373839303157
:1050000095BAED9195BAFE2FFF7395BAE078E060FE
:1050100095BA099430313233343536373839303136
:10502000A5BAED91A5BAFE2FFF7395BAE078E061BD
:1050300095BA099430313233343536373839303116
:10504000A5BAED9195BAFE2FFF73A5BAE078E0629C
:1050500095BA0994303132333435363738393031F6
:10506000A5BAED9195BAFE2FFF73A5BAE078E0637B
:1050700095BA0994303132333435363738393031D6
:10508000A5BAED91A5BAFE2FFF7395BAE078E0645A
:1050900095BA0994303132333435363738393031B6
:1050A000A5BAED9195BAFE2FFF7395BAE078E06549
:1050B00095BA099430313233343536373839303196
:1050C000A5BAED9195BAFE2FFF7395BAE078E06628
:1050D00095BA099430313233343536373839303176
:1050E00095BAED9195BAFE2FFF7395BAE078E06717
:1050F00095BA099430313233343536373839303156
:1051000095BAED9195BAFE2FFF7395BAE078E060FD
:1051100095BA099430313233343536373839303135
:1051200095BAED91A5BAFE2FFF7395BAE078E061CC
:1051300095BA099430313233343536373839303115
:10514000A5BAED9195BAFE2FFF73A5BAE078E0629B
:1051500095BA0994303132333435363738393031F5
:10516000A5BAED9195BAFE2FFF73A5BAE078E0637A
:1051700095BA0994303132333435363738393031D5
:10518000A5BAED9195BAFE2FFF73A5BAE078E06459
:1051900095BA0994303132333435363738393031B5
:1051A000A5BAED91A5BAFE2FFF73A5BAE078E06528
:1051B00095BA099430313233343536373839303195
:1051C00095BAED91A5BAFE2FFF73A5BAE078E06617
:1051D00095BA099430313233343536373839303175
:1051E00095BAED9195BAFE2FFF7395BAE078E06716
:1051F00095BA099430313233343536373839303155
:1052000095BAED9195BAFE2FFF7395BAE078E060FC
:1052100095BA099430313233343536373839303134
:10522000A5BAED91A5BAFE2FFF7395BAE078E061BB
:1052300095BA099430313233343536373839303114
:10524000A5BAED9195BAFE2FFF73A5BAE078E0629A
:1052500095BA0994303132333435363738393031F4
:10526000A5BAED9195BAFE2FFF73A5BAE078E06379
:1052700095BA0994303132333435363738393031D4
:10528000A5BAED91A5BAFE2FFF7395BAE078E06458
:1052900095BA0994303132333435363738393031B4
:1052A000A5BAED91A5BAFE2FFF7395BAE078E06537
:1052B00095BA099430313233343536373839303194
:1052C000A5BAED9195BAFE2FFF73A5BAE078E06616
:1052D00095BA099430313233343536373839303174
:1052E00095BAED9195BAFE2FFF7395BAE078E06715
:1052F00095BA099430313233343536373839303154
:1053000095BAED9195BAFE2FFF7395BAE078E060FB
:1053100095BA099430313233343536373839303133
:1053200095BAED91A5BAFE2FFF73A5BAE078E061BA
:1053300095BA099430313233343536373839303113
:10534000A5BAED9195BAFE2FFF7395BAE078E062A9
:1053500095BA0994303132333435363738393031F3
:1053600095BAED91A5BAFE2FFF7395BAE078E06388
:1053700095BA0994303132333435363738393031D3
:1053800095BAED9195BAFE2FFF73A5BAE078E06467
:1053900095BA0994303132333435363738393031B3
:1053A00095BAED9195BAFE2FFF73A5BAE078E06546
:1053B00095BA099430313233343536373839303193
:1053C000A5BAED91A5BAFE2FFF7395BAE078E06615
:1053D00095BA099430313233343536373839303173
:1053E00095BAED9195BAFE2FFF7395BAE078E06714
:1053F00095BA099430313233343536373839303153
:1054000095BAED9195BAFE2FFF7395BAE078E060FA
:1054100095BA099430313233343536373839303132
:10542000A5BAED91A5BAFE2FFF73A5BAE078E061A9
:1054300095BA099430313233343536373839303112
:1054400095BAED91A5BAFE2FFF7395BAE078E062A8
:1054500095BA0994303132333435363738393031F2
:1054600095BAED91A5BAFE2FFF7395BAE078E06387
:1054700095BA0994303132333435363738393031D2
:1054800095BAED91A5BAFE2FFF7395BAE078E06466
:1054900095BA0994303132333435363738393031B2
:1054A00095BAED91A5BAFE2FFF7395BAE078E06545
:1054B00095BA099430313233343536373839303192
:1054C00095BAED91A5BAFE2FFF7395BAE078E06624
:1054D00095BA099430313233343536373839303172
:1054E00095BAED9195BAFE2FFF7395BAE078E06713
:1054F00095BA099430313233343536373839303152
:1055000095BAED9195BAFE2FFF7395BAE078E060F9
:1055100095BA099430313233343536373839303131
:10552000A5BAED9195BAFE2FFF73A5BAE078E061B8
:1055300095BA099430313233343536373839303111
:10554000A5BAED9195BAFE2FFF73A5BAE078E06297
:1055500095BA0994303132333435363738393031F1
:10556000A5BAED9195BAFE2FFF73A5BAE078E06376
:1055700095BA0994303132333435363738393031D1
:10558000A5BAED9195BAFE2FFF73A5BAE078E06455
:1055900095BA0994303132333435363738393031B1
:1055A000A5BAED9195BAFE2FFF73A5BAE078E06534
:1055B00095BA099430313233343536373839303191
:1055C00095BAED91A5BAFE2FFF7395BAE078E06623
:1055D00095BA099430313233343536373839303171
:1055E00095BAED9195BAFE2FFF7395BAE078E06712
:1055F00095BA099430313233343536373839303151
:1056000095BAED9195BAFE2FFF7395BAE078E060F8
:1056100095BA099430313233343536373839303130
:10562000A5BAED9195BAFE2FFF73A5BAE078E061B7
:1056300095BA099430313233343536373839303110
:10564000A5BAED9195BAFE2FFF73A5BAE078E06296
:1056500095BA0994303132333435363738393031F0
:10566000A5BAED9195BAFE2FFF73A5BAE078E06375
:1056700095BA0994303132333435363738393031D0
:10568000A5BAED9195BAFE2FFF73A5BAE078E06454
:1056900095BA0994303132333435363738393031B0
:1056A00095BAED91A5BAFE2FFF7395BAE078E06543
:1056B00095BA099430313233343536373839303190
:1056C00095BAED91A5BAFE2FFF7395BAE078E06622
:1056D00095BA099430313233343536373839303170
:1056E00095BAED9195BAFE2FFF7395BAE078E06711
:1056F00095BA099430313233343536373839303150
:1057000095BAED9195BAFE2FFF7395BAE078E060F7
:1057100095BA09943031323334353637383930312F
:10572000A5BAED9195BAFE2FFF73A5BAE078E061B6
:1057300095BA09943031323334353637383930310F
:10574000A5BAED9195BAFE2FFF73A5BAE078E06295
:1057500095BA0994303132333435363738393031EF
:10576000A5BAED9195BAFE2FFF73A5BAE078E06374
:1057700095BA0994303132333435363738393031CF
:10578000A5BAED91A5BAFE2FFF73A5BAE078E06443
:1057900095BA0994303132333435363738393031AF
:1057A000A5BAED91A5BAFE2FFF73A5BAE078E06522
:1057B00095BA09943031323334353637383930318F
:1057C000A5BAED9195BAFE2FFF73A5BAE078E06611
:1057D00095BA09943031323334353637383930316F
:1057E00095BAED9195BAFE2FFF7395BAE078E06710
:1057F00095BA09943031323334353637383930314F
:1058000095BAED9195BAFE2FFF7395BAE078E060F6
:1058100095BA09943031323334353637383930312E
:10582000A5BAED9195BAFE2FFF73A5BAE078E061B5
:1058300095BA09943031323334353637383930310E
:10584000A5BAED9195BAFE2FFF73A5BAE078E06294
:1058500095BA0994303132333435363738393031EE
:1058600095BAED91A5BAFE2FFF7395BAE078E06383
:1058700095BA0994303132333435363738393031CE
:1058800095BAED91A5BAFE2FFF7395BAE078E06462
:1058900095BA0994303132333435363738393031AE
:1058A000A5BAED9195BAFE2FFF73A5BAE078E06531
:1058B00095BA09943031323334353637383930318E
:1058C000A5BAED9195BAFE2FFF73A5BAE078E06610
:1058D00095BA09943031323334353637383930316E
:1058E00095BAED9195BAFE2FFF7395BAE078E0670F
:1058F00095BA09943031323334353637383930314E
:1059000095BAED9195BAFE2FFF7395BAE078E060F5
:1059100095BA09943031323334353637383930312D
:10592000A5BAED9195BAFE2FFF73A5BAE078E061B4
:1059300095BA09943031323334353637383930310D
:10594000A5BAED9195BAFE2FFF73A5BAE078E06293
:1059500095BA0994303132333435363738393031ED
:10596000A5BAED9195BAFE2FFF73A5BAE078E06372
:1059700095BA0994303132333435363738393031CD
:1059800095BAED91A5BAFE2FFF7395BAE078E06461
:1059900095BA0994303132333435363738393031AD
:1059A00095BAED91A5BAFE2FFF7395BAE078E06540
:1059B00095BA09943031323334353637383930318D
:1059C00095BAED91A5BAFE2FFF7395BAE078E0661F
:1059D00095BA09943031323334353637383930316D
:1059E00095BAED9195BAFE2FFF7395BAE078E0670E
:1059F00095BA09943031323334353637383930314D
:105A000095BAED9195BAFE2FFF7395BAE078E060F4
:105A100095BA09943031323334353637383930312C
:105A2000A5BAED91A5BAFE2FFF73A5BAE078E061A3
:105A300095BA09943031323334353637383930310C
:105A400095BAED9195BAFE2FFF73A5BAE078E062A2
:105A500095BA0994303132333435363738393031EC
:105A600095BAED91A5BAFE2FFF7395BAE078E06381
:105A700095BA0994303132333435363738393031CC
:105A800095BAED91A5BAFE2FFF7395BAE078E06460
:105A900095BA0994303132333435363738393031AC
:105AA000A5BAED9195BAFE2FFF7395BAE078E0653F
:105AB00095BA09943031323334353637383930318C
:105AC000A5BAED91A5BAFE2FFF73A5BAE078E066FE
:105AD00095BA09943031323334353637383930316C
:105AE00095BAED9195BAFE2FFF7395BAE078E0670D
:105AF00095BA09943031323334353637383930314C
:105B000095BAED9195BAFE2FFF7395BAE078E060F3
:105B100095BA09943031323334353637383930312B
:105B200095BAED91A5BAFE2FFF73A5BAE078E061B2
:105B300095BA09943031323334353637383930310B
:105B400095BAED91A5BAFE2FFF7395BAE078E062A1
:105B500095BA0994303132333435363738393031EB
:105B600095BAED91A5BAFE2FFF7395BAE078E06380
:105B700095BA0994303132333435363738393031CB
:105B800095BAED91A5BAFE2FFF7395BAE078E0645F
:105B900095BA0994303132333435363738393031AB
:105BA00095BAED91A5BAFE2FFF7395BAE078E0653E
:105BB00095BA09943031323334353637383930318B
:105BC00095BAED91A5BAFE2FFF73A5BAE078E0660D
:105BD00095BA09943031323334353637383930316B
:105BE00095BAED9195BAFE2FFF7395BAE078E0670C
:105BF00095BA09943031323334353637383930314B
:105C000095BAED9195BAFE2FFF7395BAE078E060F2
:105C100095BA09943031323334353637383930312A
:105C2000A5BAED9195BAFE2FFF7395BAE078E061C1
:105C300095BA09943031323334353637383930310A
:105C4000A5BAED9195BAFE2FFF7395BAE078E062A0
:105C500095BA0994303132333435363738393031EA
:105C600095BAED91A5BAFE2FFF7395BAE078E0637F
:105C700095BA0994303132333435363738393031CA
:105C800095BAED91A5BAFE2FFF7395BAE078E0645E
:105C900095BA0994303132333435363738393031AA
:105CA00095BAED9195BAFE2FFF73A5BAE078E0653D
:105CB00095BA09943031323334353637383930318A
:105CC00095BAED9195BAFE2FFF73A5BAE078E0661C
:105CD00095BA09943031323334353637383930316A
:105CE00095BAED9195BAFE2FFF7395BAE078E0670B
:105CF00095BA09943031323334353637383930314A
:105D000095BAED9195BAFE2FFF7395BAE078E060F1
:105D100095BA099430313233343536373839303129
:105D2000A5BAED91A5BAFE2FFF7395BAE078E061B0
:105D300095BA099430313233343536373839303109
:105D400095BAED91A5BAFE2FFF7395BAE078E0629F
:105D500095BA0994303132333435363738393031E9
:105D600095BAED91A5BAFE2FFF7395BAE078E0637E
:105D700095BA0994303132333435363738393031C9
:105D800095BAED91A5BAFE2FFF7395BAE078E0645D
:105D900095BA0994303132333435363738393031A9
:105DA00095BAED91A5BAFE2FFF7395BAE078E0653C
:105DB00095BA099430313233343536373839303189
:105DC000A5BAED91A5BAFE2FFF7395BAE078E0660B
:105DD00095BA099430313233343536373839303169
:105DE00095BAED9195BAFE2FFF7395BAE078E0670A
:105DF00095BA099430313233343536373839303149
:105E000095BAED9195BAFE2FFF7395BAE078E060F0
:105E100095BA099430313233343536373839303128
:105E200095BAED91A5BAFE2FFF7395BAE078E061BF
:105E300095BA099430313233343536373839303108
:105E4000A5BAED9195BAFE2FFF73A5BAE078E0628E
:105E500095BA0994303132333435363738393031E8
:105E600095BAED9195BAFE2FFF7395BAE078E0638D
:105E700095BA0994303132333435363738393031C8
:105E800095BAED9195BAFE2FFF7395BAE078E0646C
:105E900095BA0994303132333435363738393031A8
:105EA00095BAED9195BAFE2FFF7395BAE078E0654B
:105EB00095BA099430313233343536373839303188
:105EC00095BAED9195BAFE2FFF7395BAE078E0662A
:105ED00095BA099430313233343536373839303168
:105EE00095BAED9195BAFE2FFF7395BAE078E06709
:105EF00095BA099430313233343536373839303148
:105F000095BAED9195BAFE2FFF7395BAE078E060EF
:105F100095BA099430313233343536373839303127
:105F200095BAED9195BAFE2FFF7395BAE078E061CE
:105F300095BA099430313233343536373839303107
:105F400095BAED9195BAFE2FFF7395BAE078E062AD
:105F500095BA0994303132333435363738393031E7
:105F600095BAED9195BAFE2FFF7395BAE078E0638C
:105F700095BA0994303132333435363738393031C7
:105F800095BAED9195BAFE2FFF7395BAE078E0646B
:105F900095BA0994303132333435363738393031A7
:105FA00095BAED9195BAFE2FFF7395BAE078E0654A
:105FB00095BA099430313233343536373839303187
:105FC00095BAED9195BAFE2FFF7395BAE078E06629
:105FD00095BA099430313233343536373839303167
:105FE000A5BAED91A5BAFE2FFF73A5BAE078E067D8
:105FF00095BA099430313233343536373839303147
:1060000095BAED9195BAFE2FFF7395BAE078E060EE
:1060100095BA099430313233343536373839303126
:1060200095BAED91A5BAFE2FFF7395BAE078E061BD
:1060300095BA099430313233343536373839303106
:1060400095BAED9195BAFE2FFF73A5BAE078E0629C
:1060500095BA0994303132333435363738393031E6
:1060600095BAED9195BAFE2FFF7395BAE078E0638B
:1060700095BA0994303132333435363738393031C6
:1060800095BAED9195BAFE2FFF7395BAE078E0646A
:1060900095BA0994303132333435363738393031A6
:1060A00095BAED9195BAFE2FFF7395BAE078E06549
:1060B00095BA099430313233343536373839303186
:1060C00095BAED9195BAFE2FFF7395BAE078E06628
:1060D00095BA099430313233343536373839303166
:1060E00095BAED9195BAFE2FFF7395BAE078E06707
:1060F00095BA099430313233343536373839303146
:1061000095BAED9195BAFE2FFF7395BAE078E060ED
:1061100095BA099430313233343536373839303125
:1061200095BAED9195BAFE2FFF7395BAE078E061CC
:1061300095BA099430313233343536373839303105
:1061400095BAED9195BAFE2FFF7395BAE078E062AB
:1061500095BA0994303132333435363738393031E5
:1061600095BAED91A5BAFE2FFF73A5BAE078E0636A
:1061700095BA0994303132333435363738393031C5
:10618000A5BAED9195BAFE2FFF73A5BAE078E06449
:1061900095BA0994303132333435363738393031A5
:1061A000A5BAED9195BAFE2FFF73A5BAE078E06528
:1061B00095BA099430313233343536373839303185
:1061C00095BAED91A5BAFE2FFF73A5BAE078E06607
:1061D00095BA099430313233343536373839303165
:1061E00095BAED9195BAFE2FFF7395BAE078E06706
:1061F00095BA099430313233343536373839303145
:1062000095BAED9195BAFE2FFF7395BAE078E060EC
:1062100095BA099430313233343536373839303124
:10622000A5BAED9195BAFE2FFF7395BAE078E061BB
:1062300095BA099430313233343536373839303104
:10624000A5BAED9195BAFE2FFF7395BAE078E0629A
:1062500095BA0994303132333435363738393031E4
:10626000A5BAED91A5BAFE2FFF7395BAE078E06369
:1062700095BA0994303132333435363738393031C4
:10628000A5BAED9195BAFE2FFF73A5BAE078E06448
:1062900095BA0994303132333435363738393031A4
:1062A000A5BAED9195BAFE2FFF73A5BAE078E06527
:1062B00095BA099430313233343536373839303184
:1062C000A5BAED91A5BAFE2FFF7395BAE078E06606
:1062D00095BA099430313233343536373839303164
:1062E00095BAED9195BAFE2FFF7395BAE078E06705
:1062F00095BA099430313233343536373839303144
:1063000095BAED9195BAFE2FFF7395BAE078E060EB
:1063100095BA099430313233343536373839303123
:1063200095BAED9195BAFE2FFF7395BAE078E061CA
:1063300095BA099430313233343536373839303103
:1063400095BAED9195BAFE2FFF7395BAE078E062A9
:1063500095BA0994303132333435363738393031E3
:1063600095BAED91A5BAFE2FFF73A5BAE078E06368
:1063700095BA0994303132333435363738393031C3
:10638000A5BAED9195BAFE2FFF7395BAE078E06457
:1063900095BA0994303132333435363738393031A3
:1063A000A5BAED9195BAFE2FFF7395BAE078E06536
:1063B00095BA099430313233343536373839303183
:1063C00095BAED91A5BAFE2FFF73A5BAE078E06605
:1063D00095BA099430313233343536373839303163
:1063E00095BAED9195BAFE2FFF7395BAE078E06704
:1063F00095BA099430313233343536373839303143
:1064000095BAED9195BAFE2FFF7395BAE078E060EA
:1064100095BA099430313233343536373839303122
:1064200095BAED9195BAFE2FFF73A5BAE078E061B9
:1064300095BA099430313233343536373839303102
:1064400095BAED9195BAFE2FFF73A5BAE078E06298
:1064500095BA0994303132333435363738393031E2
:1064600095BAED91A5BAFE2FFF73A5BAE078E06367
:1064700095BA0994303132333435363738393031C2
:10648000A5BAED9195BAFE2FFF73A5BAE078E06446
:1064900095BA0994303132333435363738393031A2
:1064A000A5BAED9195BAFE2FFF73A5BAE078E06525
:1064B00095BA099430313233343536373839303182
:1064C00095BAED91A5BAFE2FFF73A5BAE078E06604
:1064D00095BA099430313233343536373839303162
:1064E00095BAED9195BAFE2FFF7395BAE078E06703
:1064F00095BA099430313233343536373839303142
:1065000095BAED9195BAFE2FFF7395BAE078E060E9
:1065100095BA099430313233343536373839303121
:1065200095BAED9195BAFE2FFF7395BAE078E061C8
:1065300095BA099430313233343536373839303101
:1065400095BAED9195BAFE2FFF7395BAE078E062A7
:1065500095BA0994303132333435363738393031E1
:1065600095BAED91A5BAFE2FFF7395BAE078E06376
:1065700095BA0994303132333435363738393031C1
:10658000A5BAED9195BAFE2FFF73A5BAE078E06445
:1065900095BA0994303132333435363738393031A1
:1065A000A5BAED91A5BAFE2FFF7395BAE078E06524
:1065B00095BA099430313233343536373839303181
:1065C00095BAED91A5BAFE2FFF73A5BAE078E06603
:1065D00095BA099430313233343536373839303161
:1065E00095BAED9195BAFE2FFF7395BAE078E06702
:1065F00095BA099430313233343536373839303141
:1066000095BAED9195BAFE2FFF7395BAE078E060E8
:1066100095BA099430313233343536373839303120
:1066200095BAED9195BAFE2FFF73A5BAE078E061B7
:1066300095BA099430313233343536373839303100
:1066400095BAED91A5BAFE2FFF7395BAE078E06296
:1066500095BA0994303132333435363738393031E0
:10666000A5BAED91A5BAFE2FFF73A5BAE078E06355
:1066700095BA0994303132333435363738393031C0
:1066800095BAED91A5BAFE2FFF7395BAE078E06454
:1066900095BA0994303132333435363738393031A0
:1066A00095BAED91A5BAFE2FFF7395BAE078E06533
:1066B00095BA099430313233343536373839303180
:1066C00095BAED91A5BAFE2FFF7395BAE078E06612
:1066D00095BA099430313233343536373839303160
:1066E00095BAED9195BAFE2FFF7395BAE078E06701
:1066F00095BA099430313233343536373839303140
:1067000095BAED9195BAFE2FFF7395BAE078E060E7
:1067100095BA09943031323334353637383930311F
:1067200095BAED9195BAFE2FFF7395BAE078E061C6
:1067300095BA0994303132333435363738393031FF
:1067400095BAED9195BAFE2FFF7395BAE078E062A5
:1067500095BA0994303132333435363738393031DF
:1067600095BAED91A5BAFE2FFF73A5BAE078E06364
:1067700095BA0994303132333435363738393031BF
:10678000A5BAED9195BAFE2FFF73A5BAE078E06443
:1067900095BA09943031323334353637383930319F
:1067A00095BAED91A5BAFE2FFF73A5BAE078E06522
:1067B00095BA09943031323334353637383930317F
:1067C00095BAED9195BAFE2FFF73A5BAE078E06611
:1067D00095BA09943031323334353637383930315F
:1067E000A5BAED91A5BAFE2FFF7395BAE078E067E0
:1067F00095BA09943031323334353637383930313F
:1068000095BAED9195BAFE2FFF7395BAE078E060E6
:1068100095BA09943031323334353637383930311E
:10682000A5BAED9195BAFE2FFF7395BAE078E061B5
:1068300095BA0994303132333435363738393031FE
:10684000A5BAED9195BAFE2FFF7395BAE078E06294
:1068500095BA0994303132333435363738393031DE
:10686000A5BAED91A5BAFE2FFF7395BAE078E06363
:1068700095BA0994303132333435363738393031BE
:10688000A5BAED9195BAFE2FFF73A5BAE078E06442
:1068900095BA09943031323334353637383930319E
:1068A000A5BAED9195BAFE2FFF73A5BAE078E06521
:1068B00095BA09943031323334353637383930317E
:1068C000A5BAED9195BAFE2FFF73A5BAE078E06600
:1068D00095BA09943031323334353637383930315E
:1068E00095BAED9195BAFE2FFF7395BAE078E067FF
:1068F00095BA09943031323334353637383930313E
:1069000095BAED9195BAFE2FFF7395BAE078E060E5
:1069100095BA09943031323334353637383930311D
:1069200095BAED91A5BAFE2FFF7395BAE078E061B4
:1069300095BA0994303132333435363738393031FD
:1069400095BAED9195BAFE2FFF7395BAE078E062A3
:1069500095BA0994303132333435363738393031DD
:10696000A5BAED91A5BAFE2FFF7395BAE078E06362
:1069700095BA0994303132333435363738393031BD
:1069800095BAED91A5BAFE2FFF7395BAE078E06451
:1069900095BA09943031323334353637383930319D
:1069A00095BAED91A5BAFE2FFF7395BAE078E06530
:1069B00095BA09943031323334353637383930317D
:1069C000A5BAED91A5BAFE2FFF73A5BAE078E066EF
:1069D00095BA09943031323334353637383930315D
:1069E00095BAED9195BAFE2FFF7395BAE078E067FE
:1069F00095BA09943031323334353637383930313D
:106A000095BAED9195BAFE2FFF7395BAE078E060E4
:106A100095BA09943031323334353637383930311C
:106A200095BAED91A5BAFE2FFF7395BAE078E061B3
:106A300095BA0994303132333435363738393031FC
:106A400095BAED9195BAFE2FFF7395BAE078E062A2
:106A500095BA0994303132333435363738393031DC
:106A6000A5BAED91A5BAFE2FFF7395BAE078E06361
:106A700095BA0994303132333435363738393031BC
:106A800095BAED91A5BAFE2FFF7395BAE078E06450
:106A900095BA09943031323334353637383930319C
:106AA00095BAED91A5BAFE2FFF7395BAE078E0652F
:106AB00095BA09943031323334353637383930317C
:106AC00095BAED91A5BAFE2FFF7395BAE078E0660E
:106AD00095BA09943031323334353637383930315C
:106AE000A5BAED9195BAFE2FFF7395BAE078E067ED
:106AF00095BA09943031323334353637383930313C
:106B000095BAED9195BAFE2FFF7395BAE078E060E3
:106B100095BA09943031323334353637383930311B
:106B2000A5BAED9195BAFE2FFF7395BAE078E061B2
:106B300095BA0994303132333435363738393031FB
:106B4000A5BAED9195BAFE2FFF7395BAE078E06291
:106B500095BA0994303132333435363738393031DB
:106B6000A5BAED9195BAFE2FFF73A5BAE078E06360
:106B700095BA0994303132333435363738393031BB
:106B8000A5BAED91A5BAFE2FFF7395BAE078E0643F
:106B900095BA09943031323334353637383930319B
:106BA000A5BAED91A5BAFE2FFF7395BAE078E0651E
:106BB00095BA09943031323334353637383930317B
:106BC000A5BAED9195BAFE2FFF73A5BAE078E066FD
:106BD00095BA09943031323334353637383930315B
:106BE00095BAED9195BAFE2FFF7395BAE078E067FC
:106BF00095BA09943031323334353637383930313B
:106C000095BAED9195BAFE2FFF7395BAE078E060E2
:106C100095BA09943031323334353637383930311A
:106C2000A5BAED91A5BAFE2FFF7395BAE078E061A1
:106C300095BA0994303132333435363738393031FA
:106C400095BAED91A5BAFE2FFF7395BAE078E06290
:106C500095BA0994303132333435363738393031DA
:106C600095BAED91A5BAFE2FFF7395BAE078E0636F
:106C700095BA0994303132333435363738393031BA
:106C800095BAED91A5BAFE2FFF7395BAE078E0644E
:106C900095BA09943031323334353637383930319A
:106CA00095BAED91A5BAFE2FFF7395BAE078E0652D
:106CB00095BA09943031323334353637383930317A
:106CC000A5BAED91A5BAFE2FFF73A5BAE078E066EC
:106CD00095BA09943031323334353637383930315A
:106CE00095BAED9195BAFE2FFF7395BAE078E067FB
:106CF00095BA09943031323334353637383930313A
:106D000095BAED9195BAFE2FFF7395BAE078E060E1
:106D100095BA099430313233343536373839303119
:106D200095BAED9195BAFE2FFF7395BAE078E061C0
:106D300095BA0994303132333435363738393031F9
:106D400095BAED9195BAFE2FFF7395BAE078E0629F
:106D500095BA0994303132333435363738393031D9
:106D6000A5BAED91A5BAFE2FFF7395BAE078E0635E
:106D700095BA0994303132333435363738393031B9
:106D8000A5BAED91A5BAFE2FFF73A5BAE078E0642D
:106D900095BA099430313233343536373839303199
:106DA000A5BAED91A5BAFE2FFF73A5BAE078E0650C
:106DB00095BA099430313233343536373839303179
:106DC000A5BAED91A5BAFE2FFF73A5BAE078E066EB
:106DD00095BA099430313233343536373839303159
:106DE00095BAED9195BAFE2FFF7395BAE078E067FA
:106DF00095BA099430313233343536373839303139
:106E000095BAED9195BAFE2FFF7395BAE078E060E0
:106E100095BA099430313233343536373839303118
:106E200095BAED9195BAFE2FFF7395BAE078E061BF
:106E300095BA0994303132333435363738393031F8
:106E400095BAED9195BAFE2FFF7395BAE078E0629E
:106E500095BA0994303132333435363738393031D8
:106E6000A5BAED91A5BAFE2FFF7395BAE078E0635D
:106E700095BA0994303132333435363738393031B8
:106E8000A5BAED9195BAFE2FFF73A5BAE078E0643C
:106E900095BA099430313233343536373839303198
:106EA000A5BAED9195BAFE2FFF73A5BAE078E0651B
:106EB00095BA099430313233343536373839303178
:106EC000A5BAED9195BAFE2FFF73A5BAE078E066FA
:106ED00095BA099430313233343536373839303158
:106EE00095BAED9195BAFE2FFF7395BAE078E067F9
:106EF00095BA099430313233343536373839303138
:106F000095BAED9195BAFE2FFF7395BAE078E060DF
:106F100095BA099430313233343536373839303117
:106F200095BAED9195BAFE2FFF7395BAE078E061BE
:106F300095BA0994303132333435363738393031F7
:106F400095BAED9195BAFE2FFF7395BAE078E0629D
:106F500095BA0994303132333435363738393031D7
:106F600095BAED91A5BAFE2FFF7395BAE078E0636C
:106F700095BA0994303132333435363738393031B7
:106F8000A5BAED9195BAFE2FFF73A5BAE078E0643B
:106F900095BA099430313233343536373839303197
:106FA000A5BAED9195BAFE2FFF73A5BAE078E0651A
:106FB00095BA099430313233343536373839303177
:106FC00095BAED91A5BAFE2FFF7395BAE078E06609
:106FD00095BA099430313233343536373839303157
:106FE00095BAED9195BAFE2FFF7395BAE078E067F8
:106FF00095BA099430313233343536373839303137
:1070000095BAED9195BAFE2FFF7395BAE078E060DE
:1070100095BA099430313233343536373839303116
:1070200095BAED9195BAFE2FFF7395BAE078E061BD
:1070300095BA0994303132333435363738393031F6
:1070400095BAED9195BAFE2FFF7395BAE078E0629C
:1070500095BA0994303132333435363738393031D6
:10706000A5BAED91A5BAFE2FFF7395BAE078E0635B
:1070700095BA0994303132333435363738393031B6
:10708000A5BAED9195BAFE2FFF73A5BAE078E0643A
:1070900095BA099430313233343536373839303196
:1070A000A5BAED91A5BAFE2FFF7395BAE078E06519
:1070B00095BA099430313233343536373839303176
:1070C000A5BAED9195BAFE2FFF7395BAE078E06608
:1070D00095BA099430313233343536373839303156
:1070E000A5BAED9195BAFE2FFF7395BAE078E067E7
:1070F00095BA099430313233343536373839303136
:1071000095BAED9195BAFE2FFF7395BAE078E060DD
:1071100095BA099430313233343536373839303115
:1071200095BAED9195BAFE2FFF7395BAE078E061BC
:1071300095BA0994303132333435363738393031F5
:1071400095BAED9195BAFE2FFF7395BAE078E0629B
:1071500095BA0994303132333435363738393031D5
:1071600095BAED91A5BAFE2FFF73A5BAE078E0635A
:1071700095BA0994303132333435363738393031B5
:10718000A5BAED9195BAFE2FFF73A5BAE078E06439
:1071900095BA099430313233343536373839303195
:1071A00095BAED91A5BAFE2FFF73A5BAE078E06518
:1071B00095BA099430313233343536373839303175
:1071C00095BAED9195BAFE2FFF73A5BAE078E06607
:1071D00095BA099430313233343536373839303155
:1071E00095BAED9195BAFE2FFF73A5BAE078E067E6
:1071F00095BA099430313233343536373839303135
:1072000095BAED9195BAFE2FFF7395BAE078E060DC
:1072100095BA099430313233343536373839303114
:1072200095BAED9195BAFE2FFF7395BAE078E061BB
:1072300095BA0994303132333435363738393031F4
:1072400095BAED9195BAFE2FFF7395BAE078E0629A
:1072500095BA0994303132333435363738393031D4
:10726000A5BAED91A5BAFE2FFF7395BAE078E06359
:1072700095BA0994303132333435363738393031B4
:10728000A5BAED9195BAFE2FFF73A5BAE078E06438
:1072900095BA099430313233343536373839303194
:1072A000A5BAED9195BAFE2FFF7395BAE078E06527
:1072B00095BA099430313233343536373839303174
:1072C000A5BAED9195BAFE2FFF7395BAE078E06606
:1072D00095BA099430313233343536373839303154
:1072E00095BAED9195BAFE2FFF7395BAE078E067F5
:1072F00095BA099430313233343536373839303134
:1073000095BAED9195BAFE2FFF7395BAE078E060DB
:1073100095BA099430313233343536373839303113
:1073200095BAED9195BAFE2FFF7395BAE078E061BA
:1073300095BA0994303132333435363738393031F3
:1073400095BAED9195BAFE2FFF7395BAE078E06299
:1073500095BA0994303132333435363738393031D3
:1073600095BAED91A5BAFE2FFF73A5BAE078E06358
:1073700095BA0994303132333435363738393031B3
:10738000A5BAED9195BAFE2FFF7395BAE078E06447
:1073900095BA099430313233343536373839303193
:1073A00095BAED91A5BAFE2FFF73A5BAE078E06516
:1073B00095BA099430313233343536373839303173
:1073C000A5BAED91A5BAFE2FFF7395BAE078E066F5
:1073D00095BA099430313233343536373839303153
:1073E00095BAED9195BAFE2FFF7395BAE078E067F4
:1073F00095BA099430313233343536373839303133
:1074000095BAED9195BAFE2FFF7395BAE078E060DA
:1074100095BA099430313233343536373839303112
:1074200095BAED91A5BAFE2FFF7395BAE078E061A9
:1074300095BA0994303132333435363738393031F2
:1074400095BAED91A5BAFE2FFF7395BAE078E06288
:1074500095BA0994303132333435363738393031D2
:10746000A5BAED91A5BAFE2FFF73A5BAE078E06347
:1074700095BA0994303132333435363738393031B2
:1074800095BAED91A5BAFE2FFF7395BAE078E06446
:1074900095BA099430313233343536373839303192
:1074A00095BAED91A5BAFE2FFF7395BAE078E06525
:1074B00095BA099430313233343536373839303172
:1074C00095BAED9195BAFE2FFF73A5BAE078E06604
:1074D00095BA099430313233343536373839303152
:1074E00095BAED9195BAFE2FFF7395BAE078E067F3
:1074F00095BA099430313233343536373839303132
:1075000095BAED9195BAFE2FFF7395BAE078E060D9
:1075100095BA099430313233343536373839303111
:1075200095BAED9195BAFE2FFF7395BAE078E061B8
:1075300095BA0994303132333435363738393031F1
:1075400095BAED9195BAFE2FFF7395BAE078E06297
:1075500095BA0994303132333435363738393031D1
:10756000A5BAED9195BAFE2FFF73A5BAE078E06356
:1075700095BA0994303132333435363738393031B1
:10758000A5BAED9195BAFE2FFF73A5BAE078E06435
:1075900095BA099430313233343536373839303191
:1075A000A5BAED9195BAFE2FFF73A5BAE078E06514
:1075B00095BA099430313233343536373839303171
:1075C00095BAED91A5BAFE2FFF73A5BAE078E066F3
:1075D00095BA099430313233343536373839303151
:1075E00095BAED9195BAFE2FFF7395BAE078E067F2
:1075F00095BA099430313233343536373839303131
:1076000095BAED9195BAFE2FFF7395BAE078E060D8
:1076100095BA099430313233343536373839303110
:1076200095BAED9195BAFE2FFF7395BAE078E061B7
:1076300095BA0994303132333435363738393031F0
:1076400095BAED9195BAFE2FFF7395BAE078E06296
:1076500095BA0994303132333435363738393031D0
:10766000A5BAED9195BAFE2FFF73A5BAE078E06355
:1076700095BA0994303132333435363738393031B0
:10768000A5BAED9195BAFE2FFF73A5BAE078E06434
:1076900095BA099430313233343536373839303190
:1076A00095BAED91A5BAFE2FFF7395BAE078E06523
:1076B00095BA099430313233343536373839303170
:1076C00095BAED91A5BAFE2FFF7395BAE078E06602
:1076D00095BA099430313233343536373839303150
:1076E00095BAED9195BAFE2FFF7395BAE078E067F1
:1076F00095BA099430313233343536373839303130
:1077000095BAED9195BAFE2FFF7395BAE078E060D7
:1077100095BA09943031323334353637383930310F
:1077200095BAED9195BAFE2FFF7395BAE078E061B6
:1077300095BA0994303132333435363738393031EF
:1077400095BAED9195BAFE2FFF7395BAE078E06295
:1077500095BA0994303132333435363738393031CF
:10776000A5BAED9195BAFE2FFF73A5BAE078E06354
:1077700095BA0994303132333435363738393031AF
:10778000A5BAED9195BAFE2FFF73A5BAE078E06433
:1077900095BA09943031323334353637383930318F
:1077A000A5BAED91A5BAFE2FFF73A5BAE078E06502
:1077B00095BA09943031323334353637383930316F
:1077C000A5BAED91A5BAFE2FFF73A5BAE078E066E1
:1077D00095BA09943031323334353637383930314F
:1077E00095BAED9195BAFE2FFF7395BAE078E067F0
:1077F00095BA09943031323334353637383930312F
:1078000095BAED9195BAFE2FFF7395BAE078E060D6
:1078100095BA09943031323334353637383930310E
:1078200095BAED9195BAFE2FFF7395BAE078E061B5
:1078300095BA0994303132333435363738393031EE
:1078400095BAED9195BAFE2FFF7395BAE078E06294
:1078500095BA0994303132333435363738393031CE
:10786000A5BAED9195BAFE2FFF73A5BAE078E06353
:1078700095BA0994303132333435363738393031AE
:1078800095BAED91A5BAFE2FFF7395BAE078E06442
:1078900095BA09943031323334353637383930318E
:1078A00095BAED91A5BAFE2FFF7395BAE078E06521
:1078B00095BA09943031323334353637383930316E
:1078C000A5BAED9195BAFE2FFF73A5BAE078E066F0
:1078D00095BA09943031323334353637383930314E
:1078E00095BAED9195BAFE2FFF7395BAE078E067EF
:1078F00095BA09943031323334353637383930312E
:1079000095BAED9195BAFE2FFF7395BAE078E060D5
:1079100095BA09943031323334353637383930310D
:1079200095BAED9195BAFE2FFF7395BAE078E061B4
:1079300095BA0994303132333435363738393031ED
:1079400095BAED9195BAFE2FFF7395BAE078E06293
:1079500095BA0994303132333435363738393031CD
:10796000A5BAED9195BAFE2FFF73A5BAE078E06352
:1079700095BA0994303132333435363738393031AD
:10798000A5BAED9195BAFE2FFF73A5BAE078E06431
:1079900095BA09943031323334353637383930318D
:1079A00095BAED91A5BAFE2FFF73A5BAE078E06510
:1079B00095BA09943031323334353637383930316D
:1079C00095BAED9195BAFE2FFF73A5BAE078E066FF
:1079D00095BA09943031323334353637383930314D
:1079E000A5BAED91A5BAFE2FFF7395BAE078E067CE
:1079F00095BA09943031323334353637383930312D
:107A000095BAED9195BAFE2FFF7395BAE078E060D4
:107A100095BA09943031323334353637383930310C
:107A200095BAED9195BAFE2FFF7395BAE078E061B3
:107A300095BA0994303132333435363738393031EC
:107A400095BAED9195BAFE2FFF7395BAE078E06292
:107A500095BA0994303132333435363738393031CC
:107A6000A5BAED91A5BAFE2FFF73A5BAE078E06341
:107A700095BA0994303132333435363738393031AC
:107A800095BAED91A5BAFE2FFF7395BAE078E06440
:107A900095BA09943031323334353637383930318C
:107AA000A5BAED9195BAFE2FFF7395BAE078E0651F
:107AB00095BA09943031323334353637383930316C
:107AC000A5BAED91A5BAFE2FFF73A5BAE078E066DE
:107AD00095BA09943031323334353637383930314C
:107AE00095BAED9195BAFE2FFF7395BAE078E067ED
:107AF00095BA09943031323334353637383930312C
:107B000095BAED9195BAFE2FFF7395BAE078E060D3
:107B100095BA09943031323334353637383930310B
:107B200095BAED9195BAFE2FFF73A5BAE078E061A2
:107B300095BA0994303132333435363738393031EB
:107B400095BAED91A5BAFE2FFF7395BAE078E06281
:107B500095BA0994303132333435363738393031CB
:107B600095BAED91A5BAFE2FFF7395BAE078E06360
:107B700095BA0994303132333435363738393031AB
:107B8000A5BAED9195BAFE2FFF7395BAE078E0643F
:107B900095BA09943031323334353637383930318B
:107BA00095BAED91A5BAFE2FFF7395BAE078E0651E
:107BB00095BA09943031323334353637383930316B
:107BC00095BAED91A5BAFE2FFF7395BAE078E066FD
:107BD00095BA09943031323334353637383930314B
:107BE00095BAED9195BAFE2FFF73A5BAE078E067DC
:107BF00095BA09943031323334353637383930312B
:107C000095BAED9195BAFE2FFF7395BAE078E060D2
:107C100095BA09943031323334353637383930310A
:107C200095BAED91A5BAFE2FFF7395BAE078E061A1
:107C300095BA0994303132333435363738393031EA
:107C400095BAED91A5BAFE2FFF7395BAE078E06280
:107C500095BA0994303132333435363738393031CA
:107C600095BAED91A5BAFE2FFF7395BAE078E0635F
:107C700095BA0994303132333435363738393031AA
:107C800095BAED91A5BAFE2FFF7395BAE078E0643E
:107C900095BA09943031323334353637383930318A
:107CA00095BAED91A5BAFE2FFF7395BAE078E0651D
:107CB00095BA09943031323334353637383930316A
:107CC00095BAED91A5BAFE2FFF7395BAE078E066FC
:107CD00095BA09943031323334353637383930314A
:107CE00095BAED9195BAFE2FFF7395BAE078E067EB
:107CF00095BA09943031323334353637383930312A
:107D000095BAED9195BAFE2FFF7395BAE078E060D1
:107D100095BA099430313233343536373839303109
:107D2000A5BAED9195BAFE2FFF7395BAE078E061A0
:107D300095BA0994303132333435363738393031E9
:107D400095BAED91A5BAFE2FFF7395BAE078E0627F
:107D500095BA0994303132333435363738393031C9
:107D600095BAED91A5BAFE2FFF7395BAE078E0635E
:107D700095BA0994303132333435363738393031A9
:107D800095BAED9195BAFE2FFF73A5BAE078E0643D
:107D900095BA099430313233343536373839303189
:107DA00095BAED91A5BAFE2FFF7395BAE078E0651C
:107DB00095BA099430313233343536373839303169
:107DC00095BAED91A5BAFE2FFF7395BAE078E066FB
:107DD00095BA099430313233343536373839303149
:107DE000A5BAED9195BAFE2FFF7395BAE078E067DA
:107DF00095BA099430313233343536373839303129
:107E000095BAED9195BAFE2FFF7395BAE078E060D0
:107E100095BA099430313233343536373839303108
:107E200095BAED91A5BAFE2FFF73A5BAE078E0618F
:107E300095BA0994303132333435363738393031E8
:107E4000A5BAED91A5BAFE2FFF7395BAE078E0626E
:107E500095BA0994303132333435363738393031C8
:107E600095BAED9195BAFE2FFF7395BAE078E0636D
:107E700095BA0994303132333435363738393031A8
:107E800095BAED9195BAFE2FFF7395BAE078E0644C
:107E900095BA099430313233343536373839303188
:107EA00095BAED9195BAFE2FFF7395BAE078E0652B
:107EB00095BA099430313233343536373839303168
:107EC00095BAED9195BAFE2FFF7395BAE078E0660A
:107ED00095BA099430313233343536373839303148
:107EE00095BAED9195BAFE2FFF7395BAE078E067E9
:107EF00095BA099430313233343536373839303128
:107F000085BA0C9473013031323334353637383911
:107F10003031323334353637383930313233343525
:107F200085BA0C94730130313233343536373839F1
:107F30003031323334353637383930313233343505
:107F400085BA0C94730130313233343536373839D1
:107F500030313233343536373839303132333435E5
:107F600085BA0C94730130313233343536373839B1
:107F700030313233343536373839303132333435C5
:107F800085BA0C9473013031323334353637383991
:107F900030313233343536373839303132333435A5
:107FA00085BA0C9473013031323334353637383971
:107FB0003031323334353637383930313233343585
:107FC00085BA0C9473013031323334353637383951
:107FD0003031323334353637383930313233343565
:107FE00085BA0C9473013031323334353637383931
:107FF0003031323334353637383930313233343545
:00000001FF
